:100000000C94D50E0C94F90E0C94F90E0C9461100E
:100010000C94F90E0C94F90E0C94F90E0C94B31583
:100020000C94F90E0C94F90E0C94F90E0C94F90E34
:100030000C94F90E0C94F90E0C94F90E0C94F90E24
:100040000C94F90E0C94F90E0C94F90E0C94F90E14
:100050000C94F90E0314031403140314031403146F
:1000600003140314031403140314031403140314D8
:10007000031403140314A213A5130314AB13AF1337
:10008000B313B313B313B313B313B3130114C113E3
:10009000C513C513C513C513C5130114D213D61345
:1000A000D613D613D613D613031403140314E31371
:1000B000E513E513E513E513F213F413F413F41346
:1000C000F413F413F413F4130114CE2483248624BC
:1000D00089248C248F249224952498249B249E2464
:1000E000A124A424A724AA24AD24B024B324B62494
:1000F000B924BC24BF24C224C524C824CB24006551
:100100000161007802780178006507780278037849
:100110000478006503780578006504780678006542
:1001200005780B300065067808780778006500656B
:10013000087809780A78006509780B3100650A7833
:100140000C7801610B780065016D0C7800FF0100EF
:10015000010000FFFF0000010001FF00DB080500B7
:100160000005AE080500000592080500000582089C
:10017000050000056D080F3608026D0812360805E7
:1001800036080500000A6D080A6D080A36080200E4
:100190000003360802000003360802000003360898
:1001A000026D08079208076D080CDB080400000ABE
:1001B0006D08046D080400000ADB080436400A00DC
:1001C000000A6D08056D080A00000A3640056D0832
:1001D000050000056D08050000056D080500000517
:1001E0006D0814000032360805000032360805009C
:1001F00000323608050000323608050000326D086E
:100200000800000A3608056D0805DB400600000FEF
:10021000DB400600000FDB4006DB4008EB077F09F0
:10022000AE09DD090C0A470A820ABD0AF80A330B37
:100230006E0BB80B020C4C0C960CE00C2A0D740DD6
:10024000BE0D080E200E270E430E5F0E810EA30E6C
:10025000C50EE70E090F2B0F4D0F6F0F910FB30F48
:10026000D50FF70F19103B105D107F10A1101580EE
:10027000C0E0F0E0C0800000000000000080C0E0AE
:10028000F0E0C080000103070F1FBFFFFEFCF8FC79
:10029000FEFFBF1F0F070301002070F8FCFE7F3F29
:1002A0001F0F0703070F1F3F7FFEFCF870200000A1
:1002B000000100000000000000000000000000013C
:1002C0000000000B0000F0F8F8F8F8F8F00000006B
:1002D000000307070707070300000000FCFEFEFEFF
:1002E000FEFEFC0000000000010101010100000011
:1002F0001600001F1F1F1F1F1F1F1F3F3F7EFEFCFA
:10030000FCF8F0E0C0000000C0F0F8F8FCFCFCFCD9
:100310007C7C7C7878F3FFFFFFFFFFFFF87FFFFF17
:10032000FFFFFFFFC1000000000000C0FFFFFFFF54
:10033000FFFF3F000103070F1F1F3F3F3E3E3E3EB2
:100340003F3F1F1F0F0703010017C0F0F8FCFEFE20
:10035000FE7F3F1F1F1F1F1F3F7FFEFEFCFCF8F0AC
:10036000C0071F3F3F7FFFFFF0E0E0E0E0F0F0F864
:10037000FCFFFFFF7F3F1F0700F8FCFEFFFFFFFFB2
:100380001F0F0707030307FFFFFFFEFCF8F0000045
:100390000103070F1F1F1F3F3E3E3E3E3E3F3F1FD4
:1003A0001F0F0F070100150000030F3FFFFFFFFFA6
:1003B000FEF8E080000000000000000000000000E7
:1003C0000000030F3FFFFFFFFFFEF8E0800000008A
:1003D0000000000000000000000000030F3FFFFFCE
:1003E000FFFFFEF8E0803F3F3F3F3F3F3F3F3F3F43
:1003F0003F3F3F3F3F3F3F3F3F3F3F1600C0F0F88A
:10040000FCFEFEFF3F1F1F1F1F3F7FFEFEFCFCF890
:10041000E080FEFFFFFFFFFFFFC08080808080C084
:10042000E0FFFFFFFFFFFF3F073FFFFFFFFFFFF37F
:10043000C7870F0F0F0F0F0F0707070300000000FC
:10044000000103070F0F1F1F1F3F3E3E3E3E3E3E73
:100450003E3E000015FCFE7E7E7F3F3F3F3F3F3F1C
:100460007F7FFFFEFEFCFCF8E08000E0E0E0C0C023
:10047000C0C0C0C0C0E0E0F0FFFFFFFFFF7F3F0053
:10048000FFFFFFFFFFFFFF0707070707070703033C
:1004900001010000003F3F3F3F3F3F3F3E3E3E3EA9
:1004A0003E3E3E3E3E3E3E3E001600000000000046
:1004B0000000000000FFFFFFFFFFFFFF0000000043
:1004C000F8F8F8F8F8F8F8F8F8F8F8FFFFFFFFFF89
:1004D000FFFFF8F8F8F8FFFFFFFFFFFFFF00000045
:1004E00000FFFFFFFFFFFFFF000000003F3F3F3F17
:1004F0003F3F3F0000000001010101010101000038
:10050000000015FCFE7E7E7F3F3F3F3F3F3F3F7F29
:10051000FFFEFEFCFCF8F0C0000000000000E0E080
:10052000E0E0E0E0F0F0FFFF7F7F3F1F0F00C0C082
:1005300080800003030303038787FFFFFFFFFEFCA8
:10054000F000000F1F1F1F3F3F3F3F3F3F3F3F3F18
:100550001F1F1F0F070100151F3F3F7FFFFFFFFFFA
:10056000FFFFDF9F1F1F1F1F1F1F1F1F1F000000F8
:1005700000000103070F1F3F7FFFFEFCF8F0E08043
:10058000000000C0C0808000000000000080C1FFAB
:10059000FFFFFFFFFFFC00000F1F1F1F3F3F3F3FFC
:1005A0003F3F3F3F3F1F1F0F0F03000013001F1F60
:1005B0001F1F1FFFFFFFFFFFFFFF1F1F1F1F1F004A
:1005C000000000000000FFFFFFFFFFFFFF00000032
:1005D00000000000E0E0E0E0E0FFFFFFFFFFFFFFC2
:1005E0000000000000000003030307071F3F3F3F18
:1005F0003F3F3F0000000000001500C0F0FCFCFE83
:10060000FEFF3F1F1F1F3FFFFEFEFCFCF0E000FE51
:10061000FFFFFFFFFFFF00000000000000FFFFFFE3
:10062000FFFFFFFE1FFFFFFFFFFFFFC000000000F6
:1006300000C0FFFFFFFFFFFF1F0001030F0F1F1F81
:100640003F3F3E3E3E3F3F1F1F0F0F030000C310C2
:10065000CC10D110DC10EB10FA1009111A111F1177
:1006600026112D113C1147114E1159115E116911BE
:10067000781183119211A111B011BF11CE11DD11AA
:10068000EC11FB110012071212121B122612351266
:10069000481257126612751284129312A212B112E6
:1006A000C012C512D412E512F21205131613271345
:1006B0003613471358136713781387139813AD1322
:1006C000BC13CD13DC13E313EE13F51302140F1454
:1006D0001614231430143D144A14571460146D1466
:1006E0007A147F14861493149814A914B614C3149E
:1006F000D014DD14E814F314FC140915161529158B
:1007000036154315501559155E15671506F8FC0486
:1007100004FCFC0B0B00000B0B06F8FC0404FCF8BB
:10072000090B02020B0906387C4444FCFC000A0A4F
:10073000020B0907FFFF000404FCF80F1F10111F34
:100740000F0007F8FC040404FCF85F5F0000005F82
:100750005F071830E0C0E03018060301000103060F
:1007600008F8FC04040404FCF84F5F101010105F3C
:100770004F07FCFC808080FCFC4F5F1010105F4F27
:100780000DC0F8ECC48E1E3E1E8EC4ECF8C0010FE6
:100790001B11383C3E3C38111B0F010640404040C5
:1007A00040400E1F11111F0E03C0C0C00101010502
:1007B0001010D01010010107010106000000000018
:1007C000000030784878300AE010C8E828286848E7
:1007D00010E00304090B0A0A0B09040307FC0404D4
:1007E000040404FC1F10101010101F432C00000004
:1007F00000000000000000000000000000E0C0C099
:1008000080800000000000008080808080808080E8
:100810008080800010183C3E7F0000000080800037
:1008200000000000102060C0808000000000000078
:100830000000000080C0603010000080C060000038
:100840000007C7E170381C0E06078383C3C1C1C10E
:10085000E1C1C3C3C387070F1F3EFCFCF8F0C00013
:10086000000001020E1C78F0C000000103071E7C8E
:10087000F8E080E0F8FE3F03000080F8FE1F030070
:100880000000000000000000E0F8FC3E07030181CA
:10089000E0E0700000000103FFFFFE00000003FF26
:1008A000FFFF7F00000000000000FFFF3E0000008F
:1008B000000000FFFF3F0F3FFFF8C00000000F3FA8
:1008C0007EF0C000000000000000031F7FFFFCE07E
:1008D000C08003070F0C0C0C0C0E07038180C0E0D6
:1008E000703E1F0F03C0E0F8FCE000080E0301009B
:1008F000000020100C070300000000000103070C9B
:100900001810200000010102040000003EFEFCF867
:10091000F0F1E1E3C3C7C7C6C6C606060607030370
:1009200061F1F0F8F8FCFEFF7F7FFF0F030000008D
:1009300000000000000000000000000000000000B7
:1009400000000000000000000000000000000000A7
:1009500000010F0707070707070301010000000058
:100960000000000000000101000000000000000085
:100970000000000000000000000000000000000F68
:1009800016000000000FFFFFFFFFFF0F0000000038
:100990000000000000000FFF0F000000000000003A
:1009A00000000000000000000000000000000F1622
:1009B000000000000FFFFFFFFFFF0F00000000E03E
:1009C00018C43208000FFF0F000832C418E00106F7
:1009D000081314242828282414130806010F1600CD
:1009E0000000000FFFFFFFFFFF0F000000000000EE
:1009F000D8D800000FFF0F0000000000001C3C31A1
:100A0000313F1E0000000000000000001312000033
:100A1000000080808080C0C0808080808080808056
:100A200000000000000000031F7FFFFFFFFF7F1F8B
:100A300003000000000000000000000000000101B1
:100A4000000000000000001312000000C0C0C0C081
:100A5000E0F0E0C0C0C0C0C0C0C0C0C00000000026
:100A600000011F7FFFFFFFFFFFFF7F1F010000004E
:100A70000000000000000000010101010000000072
:100A80000000131200006060E0E0F0F8F8F0E0E031
:100A9000E0E0E0E0E0606000000000000F7FFFFFAA
:100AA000FFFFFFFFFF7F0F000000000000000000BD
:100AB000000001010301010000000000001312000A
:100AC000303070F0FCFEFEFCF0F0F0F0F0F0F07072
:100AD000303000000000077FFFFFFFFFFFFFFFFF38
:100AE0007F07000000000000000000000101030378
:100AF00001010000000000001312181838F8FCFF74
:100B0000FFFFFCF8F8F8F8F8F8F8381818000000BB
:100B1000077FFFFFFFFFFFFFFFFFFF7F07000000D2
:100B200000000000000001010303030101000000B8
:100B3000000000131200323468D0AC5EBE7CF0704E
:100B4000B050A0D0E874323000000080472FD7EAC0
:100B5000F5FAF5EAD7AF5F87000000000201000058
:100B6000000001010303010100000001020012194D
:100B7000387C7C7C7C7CF9010181C1C1C1C2C2840A
:100B800018E0803F00000000FF80C07B07070707D8
:100B900007FF00FF070030408080030301000000D2
:100BA00000808047300F00000000000001010101BB
:100BB00001010100000000001219F8F8F8F8F20233
:100BC0000101818181818102020418E000FE0000A0
:100BD000FF0080F70F0F0F0F0FFF000000FF000F47
:100BE0003040878703000000000000BF9040300FB6
:100BF00000000000000001010101010101000000EE
:100C000000001219F0F0E00402028181818181016B
:100C10000102E2C418E00101FF0000E70F0F0F0F0F
:100C20000FFF0000000100FF00002F4E8781000031
:100C30000000007F30B88F40300F0000000000003F
:100C400001010101010101000000000012198020D2
:100C50001884C2C2C1C1C181010181C2C2C418E0ED
:100C6000FF0000830707070707FF00008307070748
:100C700000FF3F381C4780800000003F381C078081
:100C80008040300F0000000000000101010101015F
:100C9000010000000000121900E0F0F4F2F2F1E1AE
:100CA000010101818182828418E07E00010101013D
:100CB00001FF0000E70F0F0F0F0F00FF380F20405C
:100CC0008080000F0E07010000808040300F000080
:100CD000000000000101010101010100000000000D
:100CE0001219F8F8F8F8FAF2010101818181818284
:100CF000020418E000FE000000FF0000E70F0F0FE5
:100D00000F0FFF0000FF000F3040808F0E07010023
:100D1000000000809F40300F000000000000010133
:100D20000101010101000000000012197C7C7CF827
:100D3000000281C1C1C1C1C18102020418E000FFEB
:100D400000FF80C07B0707070707FF00008000FF48
:100D5000000F304383810000000000003FB89C4733
:100D6000300F00000000000001010101010101003D
:100D7000000000001219F8F00004E2F2F1F1F1F1C4
:100D8000E1010172F2C418E000FF0080F0010101EE
:100D90000101FF0000E0000000FF000737438080F2
:100DA000000000000F0E07818040300F000000009F
:100DB0000000010101010101010000000000121901
:100DC000000070F8FAFAF9F9F10101E1F1F2F2C468
:100DD00018E0000FE00000000000FF0080F00101BB
:100DE000010100FF0E07314080800000070703006B
:100DF00000808040300F0000000000000101010170
:100E000001010100000000000B0BF8F8F8F8F8FFF2
:100E1000FEFCF87020000000000007030100000045
:100E20000505040E1F0E040D0CFEFF0363331B3378
:100E300063C38303FFFE070F0C0C0C0C0C0C0C0D92
:100E40000C0F070D0CFEFF0303030303030303034F
:100E5000FFFE070F0C0C0C0C0C0C0C0C0C0F0710ED
:100E600010E0F8DC9E1E0F0F1F1F1F1F1E9EDCF8D8
:100E7000E0071F3F7F78E0E0C0C0E0E0787F3F1FE1
:100E8000071010E0F8FCFEFEFFFFFFFFFFFFFEFE75
:100E9000FCF8E0071F3F7F7FFFFFFFFFFFFF7F7F23
:100EA0003F1F071010E0F8FCFEFEFFFFFFFFFFFFF3
:100EB000FEFEFCF8E0071F3F7F7FFFFFFF81879F5B
:100EC0007F7F3F1F071010E0F8FCFEFEFFFFFFFFD3
:100ED000FFFFFEFEFCF8E0071F3F7F7FFFFFFF8163
:100EE00083874F5F3F1F071010E0F8FCFEFEFFFFF7
:100EF000FFFFFFFFFEFEFCF8E0071F3F7F7FFFFFC5
:100F0000FF8080814143231F071010E0F8FCFEFEA4
:100F1000FFFFFFFFFFFFFEFEFCF8E0071F3F7F7FA4
:100F2000FFFFFF80808040402018071010E0F8FC91
:100F3000FEFEFFFFFFFFFF7F7E3E3C18E0071F3FE6
:100F40007F7FFFFFFF80808040402018071010E067
:100F5000F8FCFEFEFFFFFFFF7F3F1E0E0418E007B8
:100F60001F3F7F7FFFFFFF808080404020180710D9
:100F700010E0F8FCFEFEFFFFFF3F0F010202041825
:100F8000E0071F3F7F7FFFFFFF80808040402018E9
:100F9000071010E0F8FCFEFEFFFFFF010101020256
:100FA0000418E0071F3F7F7FFFFFFF8080804040E5
:100FB0002018071010E0F8FCFEFEF1C1010101014C
:100FC00002020418E0071F3F7F7FFFFFFF80808041
:100FD00040402018071010E0F8FCF2E2C181010146
:100FE000010102020418E0071F3F7F7FFFFFFF801F
:100FF000808040402018071010E0F8C4C2828101B0
:101000000101010102020418E0071F3F7F7FFFFF7B
:10101000FF80808040402018071010E01804020272
:1010200001010101010102020418E0071F3F7F7F57
:10103000FFFFFF80808040402018071010E0180458
:10104000020201010101010102020418E007183C3B
:101050007C7EFEFFFF80808040402018071010E05B
:101060001804020201010101010102020418E00753
:1010700018207078FCFEFF80808040402018071008
:1010800010E018040202010101010101020204182A
:10109000E00718204040E0FCFF808080404020189E
:1010A000071010E01804020201010101010102020F
:1010B0000418E007182040408080808080804040F5
:1010C00020180704000000000000000002ECEC1FE4
:1010D0001F0500000000001C1C001C1C07A0FCFCDD
:1010E000A0FCFCA00007070007070007088C84FF8E
:1010F00084FC780F1F103F10180807041C70C018DC
:1011000024180C120C01071C100878FCC4EC387869
:10111000CC040F1F101F0F0000000200001C1C0356
:10112000F8FE03030F180303FEF8180F03074058D7
:10113000F0E0F0584000030100010300058080E06A
:101140008080000003000003020E0C0000000580F8
:10115000808080800000000000020C0C0000051C54
:10116000FCE000000000071F1807F8FC040404FC62
:10117000F80F1F1010101F0F050004FCFC04040CD6
:101180001F1F00073C7C44C48484040C1C101010F6
:101190001F0F07080C848484FC7808181010101F97
:1011A0000F07C0C04040FCFC401F1F0000070700A5
:1011B00007888C040404FCF81F1F1111111100078B
:1011C000F8FC040404FCF80F1F11111119080700A2
:1011D000003CFCC0000010101010131F1C0778FC0E
:1011E000848484FC780F1F1010101F0F07088C8454
:1011F0008484FCF80F1F1010101F0F02181803032F
:1012000003028E8C0001010580C0603018000103CC
:10121000060C04202020200101010105183060C0C7
:10122000800C060301000700006CEC8000000C1C21
:101230001010111F0E09F008E41414E41424C8035C
:1012400004090A090B08040307FCFC808080FCFCED
:101250000F1F1010101F0F07FCFC040404FCF81FE4
:101260001F1111111F0E07F8FC0404040C080F1FB6
:10127000101010180807FCFC04040CF8F01F1F10D5
:1012800010180F0707FCFC04040404041F1F1111AD
:1012900011101007FCFC00000000001F1F111111AD
:1012A000101007F8FC040484FCFC0F1F1010101829
:1012B0000807FCFC000000FCFC1F1F0101011F1FB0
:1012C00002FCFC1F1F07080C040404FCF8000000CB
:1012D00000001F1F08FCFCC06030180C041F1F0317
:1012E000060C18100006FCFC040404041F1F000078
:1012F000000009FCFC0000800000FCFC1F0F06033E
:101300000103060F1F08FCFC0080E038FCFC1F1FD7
:101310000E0300001F1F08F8FC04040404FCF80F6F
:101320001F101010101F0F07FCFC404040C0801F12
:101330001F1010101F0F08F8FC041C0C06FFF90FFB
:101340001F101010101F0F08FCFC406070D88C0498
:101350001F1F1010101F0F0007088C848484FC7856
:101360000F1F101010180808000000FCFC000000FF
:101370001010101F1F10101007F8FC040404FCF8D4
:101380001F1F0000001F1F0800C0F01C1CF0C00041
:101390001E1F010000011F1E0A00E0FC1CF0F01CD3
:1013A000FCE0001E1F0100000000011F1E071C7C46
:1013B000E080E07C1C1C1F0300031F1C0800008051
:1013C000FCFC800000181E070101071E18073C7C6A
:1013D000E4C484040410101011131F1E03FFFF0146
:1013E0003F3F20050000E0FC1C181F070000030120
:1013F000FFFF203F3F060000000000001830606043
:10140000301806020202020202000000000000037F
:1014100000000010706006387C4444FCFC000202AE
:1014200002030106FCFC0404FCF81F1F0202030176
:1014300006F8FC0404040801030202020106F8FC99
:101440000404FCFC010302021F1F06F8FC4444C410
:10145000C80103020203010400FCFC00020F1F127A
:1014600006F8FD0505FFFE01030202030306FCFC6E
:101470000000FCFC1F1F0202030102FCFC0B0B031B
:1014800001FFFE000B0B06FCFCF0980C041F1F0074
:1014900001030202FCFC1F1F08FCFC00FCFC00FC1A
:1014A000FC030302030302030106FCFC0000FCFC36
:1014B00003030202030106F8FC0404FCF801030222
:1014C00002030106FFFF0404FCF803030202030108
:1014D00006F8FC0404FFFF01030202030305FCFC01
:1014E00000000003030103030584C4E47C38010306
:1014F0000202020400F8FC04021F1F0206F8FC04AA
:1015000004FCFC03030000030306C0F01C1CF0C035
:101510000303000003030980F07C1C301C7CF08076
:10152000030300000000000303060C9CF0F09C0C79
:1015300003030000030306F8FD0505FFFE03030097
:10154000000303061C3C74E4C48402020202030389
:1015500004C0FFFF01003F3F2002FCFC1F1F0401ED
:101560003FFFC0203F3F000660C0C06060C0000079
:1015700000000000526164696F2065696E0052616D
:1015800064696F20617573005765636B65722061D4
:101590006B74697669657274202E2E2E0045726E0A
:1015A000657574207765636B656E202E202E202E66
:1015B00000206D696E202E202E202E005363686C53
:1015C000756D6D65726E3A20005765636B656E20B0
:1015D0006265656E646574202E202E202E0057658E
:1015E000636B7A65697420657272656963687400FB
:1015F0005765636B656E206E69636874206EF67460
:1016000069672C20526164696F2069737420616E70
:101610002E005765636B657220616B74697669652E
:101620007274005765636B657220616267657363EE
:1016300068616C746574005A656974FC62657273E4
:10164000636872656974756E672E20202057656324
:101650006B657220697374206E69636874206765B6
:101660007374656C6C742E005A656974FC626572E3
:1016700073636872656974756E672E2020205765E4
:10168000636B657220626C6569627420776569744A
:10169000657268696E2067657374656C6C7420612F
:1016A00075663A20005765636B65722067657374D1
:1016B000656C6C74206175663A20005765636B65D4
:1016C00072207374656C6C656E00205568722E0014
:1016D0002C20004EE463687374656E2000DC626544
:1016E000726D6F7267656E004D6F7267656E004850
:1016F00065757465000310140003101114000000D8
:1017000000130000000000000000000000100000B6
:10171000001300000000000000101400001014006E
:101720000010111400131500000313000000000046
:10173000001300000002090A0B0C0D0E0F121819FD
:101740005765726B74616700576F6368656E656E8D
:1017500064650053696C76657374657200322E207F
:10176000576569686E6163687473742E00312E204A
:10177000576569686E6163687473742E00486569A3
:101780006C69676162656E64004E696B6F6C617550
:1017900073004275DF2642657474616700416C6CAA
:1017A00065726865696C6967656E005265666F721F
:1017B0006D6174696F6E73742E0054616720642EBE
:1017C0002045696E68656974004D617269E420485E
:1017D000696D6D656C662E0046726F6E6C6569632F
:1017E000686E616D005066696E6773746D6F6E74BC
:1017F0006167005066696E677374736F6E6E7461B3
:101800006700436872697374692048696D6D656C1F
:10181000662E004D61696665696572746167004F87
:10182000737465726D6F6E746167004F7374657267
:10183000736F6E6E746167004B6172667265697476
:101840006167004772FC6E646F6E6E657273742E12
:10185000004173636865726D697474772E00466128
:1018600073746E6163687400526F73656E6D6F6E32
:1018700074616700576569626572666173746E2E84
:1018800000447265696BF66E696765004E65756A3E
:10189000616872008F1C931C9A1CA31CAC1CB71CA3
:1018A000BF1CC71CD7D73AD7D700D7D70057656317
:1018B0006B6572206E696368742067657374656C0C
:1018C0006C742E004EE46368737465722057656310
:1018D0006B7465726D696E3A2000AE2052544320DD
:1018E0004665686C657200B04300B1D7D700D7D7A2
:1018F0002E20D7D72E20D7D7D72E002E20002E204F
:10190000004A616E2E4665622E4DE4727A41707215
:101910002E4D6169204A756E694A756C694175671B
:101920002E5365702E4F6B742E4E6F762E44657A53
:101930002E004D6F44694D69446F46725361536F79
:101940000045696E7374656C6C756E67656E2062B8
:1019500065656E646574005A656974FC62657273CE
:10196000636872656974756E672E2045696E73745D
:10197000656C6C756E67656E207665726C617373ED
:10198000656E0042572C42592C42452C42422C484D
:10199000422C48482C48452C4D562C4E492C4E572D
:1019A0002C52502C534C2C534E2C53542C53482C0B
:1019B000544800542C542F572C542F532C572C5729
:1019C000462C462C310073006D696E006D696E0007
:1019D000526164696F2C5369676E616C005A75724D
:1019E000FC636B7365747A656E206175660A576572
:1019F000726B7365696E7374656C6C756E673F00AE
:101A00005568727A656974206CF6736368656E0A4E
:101A1000756E64206E65752065696E6C6573656EA4
:101A20003F005448203D0A5468FC72696E67656E39
:101A3000005348203D0A5363686C65737769672DCE
:101A4000486F6C737465696E005354203D0A53618E
:101A5000636873656E2D416E68616C7400534E202F
:101A60003D0A5361636873656E00534C203D0A5311
:101A70006161726C616E64005250203D0A5268656B
:101A8000696E6C616E642D5066616C7A004E5720F1
:101A90003D0A4E6F7264726865696E2D0A576573F0
:101AA0007466616C656E004E49203D0A4E6965643E
:101AB00065727361636873656E004D56203D0A4D13
:101AC00065636B6C656E627572672D0A566F727016
:101AD0006F6D6D65726E004845203D0A48657373F1
:101AE000656E004848203D0A48616D627572670066
:101AF0004842203D0A4272656D656E004242203DBB
:101B00000A4272616E64656E6275726700424520BA
:101B10003D0A4265726C696E004259203D0A42617D
:101B20007965726E004257203D0A426164656E2DF0
:101B30000A57FC727474656D626572670031203DEE
:101B4000204B65696E650A576965646572686F6CDC
:101B5000756E670A2845696E6D616C696729004674
:101B6000203D204E757220616E0A4665696572746B
:101B70006167656E005746203D204E757220616E8C
:101B80000A576F6368656E656E64656E0A756E648C
:101B9000204665696572746167656E0057203D2057
:101BA0004E757220616E0A576F6368656E656E646C
:101BB000656E00542F533D54E4676C69636820617F
:101BC00075DF65720A616E20576F6368656E656EBA
:101BD00064656E0A756E6420466569657274616736
:101BE000656E00542F573D54E4676C69636820614B
:101BF00075DF65720A616E20576F6368656E656E8A
:101C000064656E0A2853612F536F290054203D20CC
:101C100054E4676C6963680073006D696E006D69F8
:101C20006E0045696E7374656C6C756E67656E00E9
:101C3000CF1CDE1CEE1CFA1C051D101D1D1D2E1DCB
:101C40003E1D4B1D561D621D741D841D961D4E6547
:101C5000696E004A61005765636B6F6D6174202087
:101C6000202056312E352020202020A9203230304F
:101C70003920205265696D61722047726173626F0D
:101C80006E005A656974656D7066616E673A00D75B
:101C9000D7D7004D6F6E746167004469656E7374C9
:101CA0006167004D697474776F636800446F6E6E8E
:101CB0006572737461670046726569746167005389
:101CC000616D7374616700536F6E6E74616700536A
:101CD000656B756E64656E207A6569672E00546564
:101CE0006D702E20616E7A656967656E3A00576582
:101CF000636B656E206D69743A005765636B646150
:101D00007565723A005363686C756D6D65723A0063
:101D10005363686C752E64617565723A00456D7029
:101D2000662E205363686C756D6D65723A00456D63
:101D300070662E20416E7A656967652E3A00416EA5
:101D40007A65696765206175733A005765636B6DE5
:101D50006F6475733A0042756E6465736C616E648E
:101D60003A004665696572742E20616E7A6569670E
:101D7000656E3A005568727A656974206CF6736313
:101D800068656E00476572E474207A7572FC636B57
:101D90007365747A2E004D656EFC207665726C61F9
:101DA0007373656E202E2E2E000011241FBECFE50A
:101DB000D8E0DEBFCDBF14BE88E10FB6F89481BD78
:101DC00011BC0FBE12E0A0E6B0E0E4E7F2E702C00B
:101DD00005900D92A432B107D9F716E0A4E2B2E063
:101DE00001C01D92A73DB107E1F70E9477210C9435
:101DF00038390C940000BF92CF92DF92EF92FF929D
:101E00000F931F93DF93CF9300D0CDB7DEB7382F5A
:101E100084EA86BF89E993E09A83898389819A81DC
:101E2000892B21F481E090E09A83898389819A81CA
:101E300020E8A6E5B0E00C90022211F40197D9F752
:101E40009A83898389819A81892B09F470C081B131
:101E5000887F883009F06BC0330F316033B984E874
:101E600086BF89E993E09A83898389819A81892B46
:101E700021F481E090E09A83898389819A8120E826
:101E8000A6E5B0E00C90022211F40197D9F79A83ED
:101E9000898389819A81892B09F449C081B1887F1E
:101EA000803409F044C0FB0150E0642F70E06150C1
:101EB000704034E8B32E24ECC22E99E9E92E93E069
:101EC000F92E01E010E080E8D82E2AC0852F90E09E
:101ED000861797071CF4C6BE20E502C0B6BE28E5EB
:101EE000FA82E98289819A81892B11F41A83098304
:101EF00089819A810C900D2011F40197D9F79A836A
:101F0000898389819A81892B69F081B190E0887FEA
:101F1000907030E08217930729F483B181935F5F5B
:101F20005417A0F220E0541719F421E001C020E07A
:101F300084E986BF89E490E001970000E9F716BEC6
:101F4000822F0F900F90CF91DF911F910F91FF90F3
:101F5000EF90DF90CF90BF9008950F931F93DF9382
:101F6000CF9300D0CDB7DEB7382F142F84EA86BFC9
:101F700089E993E09A83898389819A81892B21F465
:101F800081E090E09A83898389819A8120E8A6E59F
:101F9000B0E00C90022211F40197D9F79A8389835B
:101FA00089819A81892B09F457C081B1887F883053
:101FB00009F052C0330F33B984E886BF89E993E052
:101FC0009A83898389819A81892B21F481E090E029
:101FD0009A83898389819A8120E8A6E5B0E00C90F4
:101FE000022211F40197D9F79A83898389819A8112
:101FF000892B91F181B1887F883171F5FB0130E047
:1020000004E849E953E061E070E020E81EC0808107
:1020100083B906BF5A83498389819A81892B11F438
:102020007A83698389819A810C90022211F4019745
:10203000D9F79A83898389819A81892B41F081B16B
:102040003196887F883219F43F5F311700F320E022
:10205000311719F421E001C020E084E986BF89E44A
:1020600090E001970000E9F716BE822F0F900F90C5
:10207000CF91DF911F910F910895FC012FB7F89434
:1020800090818181883031F0803439F0813039F4A9
:1020900089E101C08AE183BF03C08BE1FCCF13BE9D
:1020A0009CBF8281809336021092370227FF01C0C5
:1020B00078940895C198C4988FB9779BFECFC49A3D
:1020C00008951F920F920FB60F9211248F938FE0F5
:1020D00080933C028F910F900FBE0F901F90189528
:1020E00083E08093240208958FB7F894209125020D
:1020F0003091260287FF01C07894C90108958FB7F7
:10210000F89420913A0230913B0287FF01C0789405
:10211000C9010895DC01E7E6F0E083E001900D924B
:102120008150E1F708958091390208951F9387FD4A
:1021300080E0182F85360CF014E610938A0081E8B1
:102140000E945A10812F992787FD90952FEF30E03C
:10215000AC01429FC001439F900D529F900D1124EE
:1021600064E670E00E94EC38862F0E945A101F919E
:1021700008950F931F93082F882321F1C09889E4B5
:1021800090E001970000E9F7C09A10EB812F0E94C0
:102190005A1080E00E945A1080E10E945A10C19AA1
:1021A000C49880E01FB8779BFECF8F5F8038D1F74F
:1021B000C49A1F5F183B51F780918A000E949610C5
:1021C0008FEA01C08EEA0E945A10009339021F91D3
:1021D0000F910895FF920F931F93CF93DF938C017C
:1021E00040EBF42EE8018F2D0E945A1080E00E94EF
:1021F0005A1080E10E945A10C19AC49890E08881D8
:102200008FB9779BFECF21969F5F9038C1F7C49A14
:10221000F39400581F4F88EBF81621F7DF91CF9108
:102220001F910F91FF90089587FD80E085360CF097
:1022300084E680933802992787FD90959C01229F20
:10224000C001239F900D329F900D112467E270E032
:102250000E94EC38CB0131E06030730709F48FEF56
:1022600083BD089580913802089580917300909104
:1022700074000895809181009091820008954FB775
:10228000F894DC01EAE6F0E087E001900D928150DD
:10229000E1F747FF01C0789408954FB7F894AAE694
:1022A000B0E0FC0187E001900D928150E1F747FF1B
:1022B00001C078940895DF93CF9300D00F92CDB7EB
:1022C000DEB790E0FC01EE0FFF1FE80FF91FA3E35C
:1022D000B2E0ED59FE4F83E001900D928150E1F79D
:1022E0004091330250913402FA01859194919A837E
:1022F00089834E5F5F4FFA0184918B83CE010196F3
:102300000E943D100F900F900F90CF91DF91089594
:102310008FB7F8949091350287FF01C07894892F88
:10232000911181E008952FB7F894813041F0813008
:1023300018F08230F1F40DC08091310221C08091FB
:102340003202882351F08091310290E0882369F4B1
:102350000BC080913202882319F480E090E010C015
:102360008091310290E0811191E081E09827892FDE
:1023700007C01092320227FF01C0789481E00895CF
:1023800027FF01C0789408952FB7F894813041F069
:10239000813018F08230F1F40DC080912F0221C0FD
:1023A00080913002882351F080912F0290E08823A1
:1023B00069F40BC080913002882319F480E090E02A
:1023C00010C080912F0290E0811191E081E0982768
:1023D000892F07C01092300227FF01C0789481E056
:1023E000089527FF01C0789408959FB7F89420912D
:1023F0002E02813011F410922E0297FF01C07894C2
:10240000822F089583B380740895882311F0AE9AC3
:1024100001C0AE9885B3089580B380720895F89492
:1024200080912402882359F0F89428E088E190E014
:102430000FB6F894A89581BD0FBE21BDFFCF2FE048
:1024400088E190E00FB6F894A89581BD0FBE21BD3C
:102450008EEE8ABB1BBA8BEF87BB84E188BB80EC16
:1024600084BB15BA83E881BB9CE592BBE9E4F0E04C
:1024700031970000E9F784B7866084BF8AB780622D
:102480008ABF8BB780628BBF87E886B986B18660CA
:1024900086B988E183BF1CBE1FBC89E08EBD8EE07B
:1024A0008BBD86E68ABD89B7806189BF83E685BD1D
:1024B00013BC9DB991E09EB984E086BF12B880E557
:1024C00080B911B890932402789480E00E94B910EA
:1024D000089590E080912402813009F491E0892FE1
:1024E000089580912402813019F0833081F404C072
:1024F00084E0809324020895F89428E088E190E035
:102500000FB6F894A89581BD0FBE21BDFFCFF894FA
:1025100028E088E190E00FB6F894A89581BD0FBE41
:1025200021BDFFCFFF920F931F93DF93CF93CDB7C2
:10253000DEB727970FB6F894DEBF0FBECDBFFFB64C
:10254000F894AAE6B0E0E3E9F1E087E001900D92AB
:102550008150E1F7198288E68E010F5F1F4FB801A5
:1025600041E00E94AD0F882309F45AC088E6B80103
:1025700047E00E94FB0E882309F452C0298127FFFF
:1025800002C081E04DC0822F82958F704AE0849F07
:10259000C00111242F70280F20936C002A81822FF4
:1025A00082958F70849FC00111242F70280F209373
:1025B0006B002B81822F82958F70849FC001112424
:1025C0002F70280F20936A002D81822F82958F70A3
:1025D000849FC00111242F70280F20936D002E813D
:1025E000822F82958F70849FC00111242F70280F35
:1025F00020936E002F81822F90E08F709070805317
:10260000984F22952F70249F90011124820F931FC1
:102610009093700080936F008AE690E00E94AF195B
:10262000F7FE01C0789427960FB6F894DEBF0FBE70
:10263000CDBFCF91DF911F910F91FF9008950F9320
:102640001F93DF93CF93CDB7DEB72B970FB6F894D8
:10265000DEBF0FBECDBF9FB7F8942091660088E71C
:102660008093660097FF01C07894309167002D3603
:1026700009F047C03B3309F050C01F8280912B0204
:102680008E8380912A028D83809172008887809149
:10269000710089878091290290E08053984F9B8731
:1026A0008A87CE0105960E94AF198823B1F18091E7
:1026B0002C02882319F08D8181508D839D81892F73
:1026C00081508D8387FF06C0995E9D83CE01089659
:1026D0000E94EF189FB7F894AAE6B0E0FE01359685
:1026E00087E001900D928150E1F71092280210923C
:1026F0002702109269001092680097FF01C0789439
:102700000CC0213331F0283709F480C0203329F47C
:1027100002C091E004C090E002C090E03FEF8091E1
:102720002D02892780932D02E32FF0E0EB33F10592
:1027300008F068C0E65DFF4FEE0FFF1F0590F491B3
:10274000E02D099490932C025EC080912C02981782
:1027500009F059C057C0992309F454C054C090934C
:102760002D0210922B02992309F44DC0E32FF0E0C3
:10277000EA5BFE4F80912B029081890F80932B02A0
:1027800042C090932D0210922A029923E1F1E32F87
:10279000F0E0E25CFE4F80912A029081890F8093E5
:1027A0002A0231C090932D0210927200992359F1A0
:1027B000E32FF0E0E95CFE4F809172009081890F79
:1027C0008093720020C0109271009923E1F0E32FF2
:1027D000F0E0E25DFE4F809171009081890F80935F
:1027E000710011C010922902992369F0E32FF0E0E3
:1027F000E75DFE4F809129029081890F8093290225
:1028000002C081113FEF3F5F309367008BE790E09C
:102810000E94E321882309F477C080E687B9369ABD
:102820008CEC91E09A83898389819A81892B21F4A8
:1028300081E090E09A83898389819A8120E4A6E2ED
:10284000B0E00C90022211F00197D9F79A838983A6
:1028500089819A81892B29F125B1822F81508E3F60
:1028600000F5223318F460E070E0C1C02B3F08F09F
:10287000BCC030E084E690E0AC01249FC001259FFD
:10288000900D349F900D112488589341225330406D
:1028900035952795820F931F68EC70E00E94EC3805
:1028A000A6C0E0917500F0E0EA58FF4F8FEF8083FB
:1028B000809175008F5F80937500853011F41092C0
:1028C0007500E6E7F0E060E020E030E009C099271D
:1028D00087FD9095280F391F6F5F3196653029F07D
:1028E000808187FFF4CF662349F0C90170E00E9420
:1028F000EC38709374006093730006C080E090E839
:10290000909374008093730083E890E00E94E32129
:10291000882309F448C0809189008823F9F08CEA63
:102920008B831C828E010D5F1F4F8FE4B80142E044
:102930000E94AD0F882389F18EEE8B838FE4B8015E
:1029400041E00E94AD0F882341F18AEA8B838FE436
:10295000B80141E00E94AD0F8823F9F08FE4BE0179
:102960006D5F7F4F42E00E94FB0E90E0882309F4E8
:1029700091E090938900992381F49B8197FD04C095
:102980008C81803809F49F5F892F8E5C863928F40A
:10299000892F992787FD909502C080E090E8909359
:1029A000820080938100A895809125029091260253
:1029B000807893708038910549F08091250290913C
:1029C0002602807893708058914011F4DF9A01C0FC
:1029D000DF988BB32B960FB6F894DEBF0FBECDBF3A
:1029E000CF91DF911F910F91089564E670E0E0911F
:1029F0007500F0E0EA58FF4F60835ACFFF920F93C3
:102A00001F93DF93CF93CDB7DEB729970FB6F89416
:102A1000DEBF0FBECDBFFFB6F89419828AE690E004
:102A20000E94AF198E010F5F1F4F882309F465C004
:102A300030916C00832F6AE00E94CC38282F2295B9
:102A4000207F832F0E94CC38290F2A8330916B007E
:102A5000832F0E94CC38282F2295207F832F0E941D
:102A6000CC38290F2B8330916A00832F0E94CC38F9
:102A7000282F2295207F832F0E94CC38290F2C836A
:102A80008DE690E00E944B198D8330916D00832F6D
:102A90006AE00E94CC38282F2295207F832F0E9445
:102AA000CC38290F2E8330916E00832F0E94CC38B2
:102AB000282F2295207F832F0E94CC38290F2F8327
:102AC000E0916F00F0917000CF0164E670E00E9429
:102AD000D8386AE070E00E94D838262F2295207FEF
:102AE000CF016AE070E00E94D838280F288780E183
:102AF000898788E6B80149E005C080E88A8388E6CE
:102B0000B80142E00E94AD0FF7FE01C0789429960B
:102B10000FB6F894DEBF0FBECDBFCF91DF911F91EE
:102B20000F91FF9008959C01FB014130510521F464
:102B300060810E9427390895CB01B9010E9417399D
:102B40000895CF93DF939C01EB014130510521F4AF
:102B50000E940F39888304C0CB01B9010E94FF385D
:102B6000DF91CF9108951F920F920FB60F9211240B
:102B70000F931F932F933F934F935F936F937F9385
:102B80008F939F93AF93BF93EF93FF93DF93CF9375
:102B900000D00F92CDB7DEB780912502909126022A
:102BA0000196909326028093250280914002909195
:102BB00041020196909341028093400280569A4EC2
:102BC00021F41092410210924002009140021091B3
:102BD0004102809127029091280201969093280249
:102BE00080932702885E9340F1F41092280210929D
:102BF00027028AE690E00E94C91980913A029091DA
:102C00003B02019690933B0280933A0280913C02F2
:102C1000823020F0815080933C0205C0813019F44D
:102C200083E08093240201151105C1F480916800AE
:102C30009091690097FD05C001969093690080937B
:102C4000680080916800909169008051974234F04B
:102C500080E090E8909369008093680020B322950B
:102C60002695269523702095217080913102882326
:102C700059F0222331F480913E0290913F02009757
:102C800059F488EC90E00CC0222341F080913E0280
:102C900090913F02009711F0019702C08AE090E006
:102CA00090933F0280933E0280913E0290913F02BA
:102CB000892B29F42093310281E08093320290B372
:102CC00092959F709095917080912F02882341F08A
:102CD000992321F480913D02882341F482E309C0C5
:102CE000992331F080913D02882311F0815001C079
:102CF0008AE080933D0280913D02882329F49093DD
:102D00002F0281E080933002829B02C090E001C0DC
:102D100092E080B386958695869580958170890F1F
:102D2000E0914502F0E0EE0FFF1FEE0FFF1FE80FEE
:102D3000F11DE45BFE4F249190914402290F2093F2
:102D4000440280934502223019F02E3F61F404C002
:102D500080912E028F5F03C080912E02815080935C
:102D60002E0210924402C8016AE070E00E94D83836
:102D7000892B09F06FC080914202863091F08F302C
:102D800081F0813171F0893161F08F3551F08837F0
:102D900041F08C3D31F0CC9902C022E003C021E02B
:102DA00001C020E08091430290E0AC01440F551F28
:102DB000480F591F420F511D440F551FCA01815022
:102DC0009F4FFC01849142505F4FFA019491909380
:102DD00043028D3619F41092420207C0813619F46D
:102DE0001092420204C0883711F0809366008091EF
:102DF00042028F5F809342028091360290913702A7
:102E0000009741F101979093370280933602892B06
:102E100009F51A8219821B828091350281508093B4
:102E200035022091330230913402F9013396F09348
:102E30003402E0933302882349F0859194919A8378
:102E40008983F9013596859194918B83CE01019602
:102E50000E943D100F900F900F90CF91DF91FF9146
:102E6000EF91BF91AF919F918F917F916F915F9102
:102E70004F913F912F911F910F910F900FBE0F9087
:102E80001F901895FC01009779F08081883160F4DB
:102E900081818C3348F420E082818C3308F021E07A
:102EA00081E02827822F089580E090E00895CF9355
:102EB000DF93EC010E944217882341F088818F5FE5
:102EC0008883883119F4188281E001C080E0DF91A5
:102ED000CF910895CF93DF93EC010E94421788238E
:102EE00051F089818F5F89838C3329F41982CE0157
:102EF0000E94571701C080E0DF91CF910895CF93D2
:102F0000DF93EC010E944217882351F08A818F5F82
:102F10008A838C3329F41A82CE010E946A1701C079
:102F200080E0DF91CF910895CF93DF93EC010E9471
:102F30004217882351F08881882321F487E1888310
:102F400081E003C08150888380E0DF91CF910895B4
:102F5000CF93DF93EC010E944217882361F08981AF
:102F6000882331F48BE38983CE010E94941703C038
:102F70008150898380E0DF91CF910895DC01FB01CE
:102F8000009729F461157105E9F480E00895611551
:102F90007105D1F09C9180819817A0F08917A0F05D
:102FA00011969C9111978181981760F0891760F0B4
:102FB00012969C916281961728F080E0691728F498
:102FC00081E008958FEF089581E00895DC01FB0111
:102FD000009729F46115710511F580E008956115D8
:102FE0007105F9F012962D913C911397828193818E
:102FF00028173907A0F08217930798F011969C9133
:1030000011978181981758F0891758F09C91608129
:10301000961728F080E0691728F481E008958FEF73
:10302000089581E00895482FE92F282F392FC901ED
:10303000845A964085589C41B8F423703070232BF5
:1030400099F4842F9E2F64E670E00E94EC38892B5F
:1030500049F420E0842F9E2F60E971E00E94EC3853
:10306000892B19F421E001C020E0822F08959C01F2
:1030700001970C9718F5CB01845A964085589C41CE
:10308000E8F42230310559F4CB010E94131888234B
:1030900019F42CE130E017C02DE130E014C02430E9
:1030A000310579F02630310561F02930310549F0DC
:1030B0002B30310531F02FE130E005C020E030E861
:1030C00002C02EE130E0C90108951F93FC01009772
:1030D000E1F062817381CB01845A964085589C410E
:1030E000A0F49181892F81508C3078F410811123C4
:1030F00061F0892F90E00E94371840E0212F30E0E6
:10310000821793071CF041E001C040E0842F1F911B
:103110000895CF93DF93EC010E9465188823C9F0CE
:103120008A819B8101979B838A8388818D3129F4D1
:103130008981823011F48CE188838A819B81845A51
:10314000964038F481E08883898384EA96E09B8303
:103150008A83DF91CF910895CF93DF93EC010E9492
:1031600065188823D1F08A819B8101969B838A838D
:1031700088818D3129F48981823011F48CE1888332
:103180008A819B818952934240F08FE188838CE051
:10319000898388E293E29B838A83DF91CF910895AC
:1031A000CF93DF93EC010E9465188823A9F08981F1
:1031B000813031F48CE08983CE010E9489180CC0E3
:1031C000815089836A817B8190E00E943718982F13
:1031D0008881981708F49883DF91CF910895CF9351
:1031E000DF93EC010E9465188823B9F08881813053
:1031F00091F48981823028F48A819B81855A964096
:1032000060F0CE010E94D0186A817B81898190E0B4
:103210000E94371801C081508883DF91CF910895B3
:10322000CF93DF93EC010E9465188823A9F0898170
:103230008C3068F48F5F89836A817B8190E00E9483
:103240003718982F8881981738F4988305C081E043
:103250008983CE010E94AC18DF91CF9108951F930E
:10326000CF93DF93EC010E946518882381F01881C9
:103270001F5F18836A817B81898190E00E943718E3
:10328000811728F481E08883CE010E941019DF9114
:10329000CF911F9108950F931F93CF93DF93EC016C
:1032A0000E946518882379F10A811B81E981E33046
:1032B00010F401501040F0E0E756FE4F8081288165
:1032C00030E0280F311D200F311FC80196958795DA
:1032D00096958795280F391FC80160E971E00E9413
:1032E000D838260F371FC80164E670E00E94D8382E
:1032F000C901861B970B67E070E00E94D8380097E1
:1033000011F487E090E0DF91CF911F910F91089524
:10331000FF920F931F93CF93DF938C010E94651848
:10332000882319F4C0E0D0E813C0F801F180FA94C2
:103330008081C82FD0E00AC0F801628173818F2D8F
:1033400090E00E943718C80FD91FFA94FF20A1F708
:10335000CE01DF91CF911F910F91FF900895CF93F0
:10336000DF93EC01009781F00E944217882361F0FF
:10337000CE0103960E94651890E0882309F491E03D
:1033800081E09827892F02C080E090E0DF91CF9103
:103390000895CF93DF93EC01009741F00E947F17CF
:1033A000882321F0CE0103960E942F19DF91CF913F
:1033B0000895CF93DF93EC01009741F00E94A81786
:1033C000882321F0CE0103960E94EF18DF91CF9160
:1033D00008950F931F93CF93DF938C01EB01009718
:1033E00039F46115710511F08FEF12C080E010C043
:1033F0006115710511F481E00BC06D5F7F4F03967D
:103400000E94E617882321F4C801BE010E94BE175E
:10341000DF91CF911F910F9108951F93CF93DF9369
:10342000EC01009791F11C81812F8450863078F156
:10343000CE0103960E944B19282F873009F420E013
:10344000133081F48B81893100F190E0821B910966
:103450004997DCF02223D9F488818230B0F08230A1
:10346000B1F416C01A3089F48B81893180F090E074
:10347000821B910949975CF0222339F488818230BC
:1034800030F0823011F483E003C080E001C081E0BD
:10349000DF91CF911F910895FF920F931F93CF93C8
:1034A000DF93EC01F62E8A010C96499708F048C08C
:1034B000CA010E94AF19882309F442C01C161D06D8
:1034C000A4F4F8012081822F90E08C0F911D489781
:1034D00044F028512C0F2083C80103960E942F1915
:1034E00019C02C0FF801208315C0209799F02227CE
:1034F00033272C1B3D0BF8018081821740F4885E36
:10350000821B8083C80103960E94EF1803C0821BB0
:10351000F8018083FF20B1F0C8010E940D1A81508C
:10352000823080F4F8018081873130F01082C80148
:1035300003960E942F1906C08F5FF801808302C096
:1035400080E001C081E0DF91CF911F910F91FF904A
:103550000895FF920F931F93CF93DF93EC01F62E04
:103560008A010C964997E0F5CA010E94AF19882399
:10357000B9F1FF2041F0C8010E940D1A813011F00D
:10358000833009F42196D7FF18C0442755274C1BD8
:103590005D0BF8012081822F90E0840F911D4897E8
:1035A00044F02851240F2083C80103960E942F194C
:1035B00015C0240FF801208311C0209779F0F8017D
:1035C00080818C1740F4885E8C1B8083C801039631
:1035D0000E94EF1803C08C1BF801808381E001C0BA
:1035E00080E0DF91CF911F910F91FF900895CF93CD
:1035F000DF93EC01FB01DA018D919C91119797FF0C
:103600000DC022273327281B390B11963C932E938C
:1036100080819181821B930B9183808320813181F2
:1036200037FF0AC08D919C911197820F931F1196BD
:103630009C938E9311821082608171816C177D073B
:103640008CF42D913C911197121613065CF4260F01
:10365000371F2C173D0724F0C61BD70BCD93DC93E7
:1036600081E001C080E0DF91CF9108956F927F9259
:103670009F92AF92BF92CF92DF92EF92FF920F9301
:103680001F93CF93DF93FC015A01902E00E410E0CA
:10369000061B170B021B130BC80168E070E00E94A9
:1036A000EC387B013801620E731EC30168E070E0E4
:1036B0000E94EC386B01E701D695DC2FCC27D7951B
:1036C000C795CE0FDF1FCE5ADD4FE616F70609F07D
:1036D00042C0C30168E070E00E94EC38FC01EA558A
:1036E000FE4FC80168E070E00E94EC38DC01AA558A
:1036F000BE4FAC91A0958081A82381E0981649F037
:10370000981658F082E0981609F0D8C020E030E012
:103710001EC020E030E0A09511C020E030E005C0E0
:1037200088818A2B89932F5F3F4F2A153B05C4F36D
:10373000C5C088818A2389932F5F3F4F2A153B0597
:10374000C4F3BCC088818A2789932F5F3F4F2A1515
:103750003B05C4F3B3C0C80168E070E00E94EC38D8
:10376000FC01EA55FE4FE081E09540E850E04A193F
:103770005B0981E0981641F0981650F082E09816A7
:1037800021F520E030E01EC020E030E0E09511C0DF
:1037900020E030E005C088818E2B89932F5F3F4F5A
:1037A0002A153B05C4F311C088818E2389932F5FAE
:1037B0003F4F2A153B05C4F308C088818E278993A3
:1037C0002F5F3F4F2A153B05C4F3C40FD51F81E07F
:1037D0009816D1F0981620F082E09816D1F525C001
:1037E000B7016F5F7F4F2FEF09C0299301968A15AC
:1037F0009B05DCF3C40FD51F6F5F7F4F6C157D05F4
:1038000044F580E090E0F3CFB70107C0199201962C
:103810008A159B05DCF3C40FD51F6F5F7F4F6C15B6
:103820007D05BCF480E090E0F3CFB7010AC0888149
:10383000809589932F5F3F4F2A153B05C4F3C40F32
:10384000D51F6F5F7F4F6C157D051CF420E030E0C5
:10385000F3CFC30168E070E00E94EC38FC01EA5548
:10386000FE4FE08181E0981641F0981650F082E01A
:10387000981621F520E030E01EC020E030E0E09511
:1038800011C020E030E005C088818E2B89932F5F26
:103890003F4F2A153B05C4F311C088818E238993BD
:1038A0002F5F3F4F2A153B05C4F308C088818E2740
:1038B00089932F5F3F4F2A153B05C4F3DF91CF91CA
:1038C0001F910F91FF90EF90DF90CF90BF90AF903E
:1038D0009F907F906F9008952F923F924F925F92AA
:1038E0006F927F928F929F92AF92BF92CF92DF9210
:1038F000EF92FF920F931F93DF93CF9300D000D0EE
:10390000CDB7DEB76C01DA018C91882E992411961F
:103910008C911197482E5524E0E4F0E0E61BF70B5C
:10392000E419F509D7FC03C0AA24BB2404C0AA24C7
:10393000BB24AC18BD089601280D391D213831056E
:103940001CF4EE24FF2406C070E8E72E7FEFF72E6C
:10395000E20EF31E12964D915C9113978F0163E076
:10396000159507956A95E1F7B8017695762F662744
:10397000779567956E5A7D4F15012C0C3D1C67019C
:10398000C21AD30A20E830E0C20ED31E9E2F9770D1
:103990001C821B8234016E187F0842C04A0D5B1DD9
:1039A000FB01E20DF31DFA83E983DF01A058BF4F4D
:1039B000B50148010894811C911C23C0FA0184912F
:1039C000282F30E0092E02C0220F331F0A94E2F79D
:1039D000F8E08F16910418F48C91832B8C9317FDCB
:1039E00005C0E981FA818081822B80834F5F5F4F20
:1039F00029813A812F5F3F4F3A8329836F5F7F4F41
:103A0000119666157705D4F24E0D5F1D69817A8196
:103A10006C0D7D1D8401EB81FC813896FC83EB836A
:103A20002B813C812415350524F4083011050CF454
:103A3000B5CF0F900F900F900F90CF91DF911F9106
:103A40000F91FF90EF90DF90CF90BF90AF909F903D
:103A50008F907F906F905F904F903F902F90089540
:103A6000982F843CB9F1853C88F4803B09F1813B77
:103A700030F4893A01F18E3A09F044C028C0873BFE
:103A800001F18A3B09F1813BE9F518C08F3D71F1E5
:103A9000803E38F4873D21F18C3D29F1863D91F53A
:103AA0001CC0863F49F18C3F51F1843E59F521C03D
:103AB0002AEB37E037C027EC37E034C02FEA37E095
:103AC00031C028EA37E02EC02BE937E02BC020E8D0
:103AD00037E028C021E737E025C020E637E022C0E4
:103AE00021E537E01FC022E437E01CC023E337E0C4
:103AF00019C026E237E016C029E137E013C02CE0F8
:103B000037E010C0892F80528F3518F02CED37E048
:103B100009C0892F90E0880F991F825F994FFC019F
:103B200025913491F901849180934E028FE0809326
:103B30004F022F5F3F4F30935102209350028EE48B
:103B400092E00895853369F1863374F4823301F18C
:103B500083332CF48033C9F08133A9F513C0833348
:103B6000D1F0843381F51AC0883321F189332CF4E4
:103B70008633D1F0873339F51AC08933F1F08A33AF
:103B800011F51EC0ECEAF5E020C0E9EFF5E01DC03C
:103B9000E7E5F5E01AC0E2E0F5E017C0E9EAF4E095
:103BA00014C0E4E5F4E011C0EBEFF3E00EC0E6EA88
:103BB000F3E00BC0E9E4F3E008C0E0EFF2E005C099
:103BC000E3ECF2E002C0EEE6F2E0849180934A0278
:103BD0008EE180934B023196F0934D02E0934C02BC
:103BE0008AE492E00895EF92FF920F931F93CF9390
:103BF000DF937C018B01C0E0D0E0D801ED91FC9116
:103C00008081882301F18A30F1F0D7011396ED917C
:103C1000FC9114970995FC01D70111968C91992775
:103C200087FD90952081820F911DC80FD91FD7FF66
:103C300003C020E030E813C0F80180819181019633
:103C400091838083DACF9E011C161D0644F4D701B0
:103C500011968C91992787FD9095281B390BC901E6
:103C6000DF91CF911F910F91FF90EF900895E2E5C2
:103C7000F2E0119286E0E235F807D9F708950F9344
:103C8000DF93CF93CDB7DEB728970FB6F894DEBF9A
:103C90000FBECDBF9A8389837C836B835E834D8304
:103CA00038872F8380E890E0BE016F5F7F4FAE01C1
:103CB0004B5F5F4F0E94F71A8823B9F080E490E0D1
:103CC000BE016D5F7F4FAE01495F5F4F0E94F71AE3
:103CD000882359F06B817C814D815E812F813885ED
:103CE00089819A8100E00E94361B28960FB6F894CD
:103CF000DEBF0FBECDBFCF91DF910F9108950F931F
:103D0000DF93CF93CDB7DEB728970FB6F894DEBF19
:103D10000FBECDBF9A8389837C836B835E834D8383
:103D200038872F8380E890E0BE016F5F7F4FAE0140
:103D30004B5F5F4F0E94F71A8823B9F080E490E050
:103D4000BE016D5F7F4FAE01495F5F4F0E94F71A62
:103D5000882359F06B817C814D815E812F8138856C
:103D600089819A8101E00E94361B28960FB6F8944B
:103D7000DEBF0FBECDBFCF91DF910F9108950F939E
:103D8000DF93CF93CDB7DEB728970FB6F894DEBF99
:103D90000FBECDBF9A8389837C836B835E834D8303
:103DA00038872F8380E890E0BE016F5F7F4FAE01C0
:103DB0004B5F5F4F0E94F71A8823B9F080E490E0D0
:103DC000BE016D5F7F4FAE01495F5F4F0E94F71AE2
:103DD000882359F06B817C814D815E812F813885EC
:103DE00089819A8102E00E94361B28960FB6F894CA
:103DF000DEBF0FBECDBFCF91DF910F9108950F931E
:103E00001F93DF93CF93CDB7DEB728970FB6F89403
:103E1000DEBF0FBECDBF9A8389837C836B835E83B5
:103E20004D8338872F8357FF0CC022273327241B4D
:103E3000350B3E832D8389819A81821B930B9A8354
:103E400089838F81988597FF0CC022273327281BF1
:103E5000390B38872F838B819C81821B930B9C832A
:103E60008B8329813A81032F0095001F0027001FB3
:103E70004B815C8157FF02608D819E81280F391F25
:103E8000213831050CF404608F819885480F591F43
:103E9000413451050CF4086080E890E0BE016F5F8A
:103EA0007F4FAE014B5F5F4F0E94F71A882309F4E2
:103EB0004DC080E490E0BE016D5F7F4FAE01495F71
:103EC0005F4F0E94F71A882309F440C0102F00FFAB
:103ED0000BC06B817C812F81388589819A8141E07B
:103EE00050E000E00E94361B11FF0BC06B817C810B
:103EF0004D815E8189819A8121E030E000E00E945D
:103F0000361B12FF10C089819A812D813E81820F5C
:103F1000931F6B817C812F813885019741E050E0B0
:103F200000E00E94361B13FF11C06B817C818F81E2
:103F30009885680F791F615070404D815E8189813D
:103F40009A8121E030E000E00E94361B28960FB6EF
:103F5000F894DEBF0FBECDBFCF91DF911F910F91BF
:103F60000895CF92DF92EF92FF920F931F93CF931A
:103F7000DF93EB016A01893208F046C0682F70E0D8
:103F8000660F771F645E7D4FFB01A591B491FD0123
:103F9000F490F09246021196FD014491409347023D
:103FA0001196B0934902A0934802E1FC12C0642F1D
:103FB00070E0E3FE05C0C00ED11EC61AD70A09C0C4
:103FC000C801861B970B62E070E00E94EC38C60EB9
:103FD000D71EE0FC13C08F2D90E0E2FE05C0C20F9B
:103FE000D31FC81BD90B0AC0A901481B590BCA0112
:103FF00062E070E00E94EC38C60FD71FCE01B60118
:1040000046E452E00E946C1CDF91CF911F910F910A
:10401000FF90EF90DF90CF900895AF92BF92CF9234
:10402000DF92EF92FF920F931F93DF93CF9300D015
:10403000CDB7DEB77A8369836A017901FA0111820B
:104040001082F90111821082882331F0813009F049
:1040500046C000E910E002C00BE810E089819A81B7
:10406000892BD9F15E010894A11CB11CC801B501CE
:104070000E94F31D9C01F0E880309F0781F1F6015A
:10408000808191818217930714F431832083F70193
:1040900080819181F8012281422F552747FD50955B
:1040A0002081420F511D480F591FF7015183408352
:1040B00057FD15C0E981FA818081882321F031966E
:1040C000FA83E983D3CFF8018281992787FD909500
:1040D000481B590BF7015183408381E001C080E008
:1040E0000F900F90CF91DF911F910F91FF90EF9064
:1040F000DF90CF90BF90AF9008952F923F924F9254
:104100005F926F927F928F929F92AF92BF92CF9267
:10411000DF92EF92FF920F931F93DF93CF9300D024
:1041200000D000D0CDB7DEB72B015A0139019E2D4A
:104130007601882341F0813009F0BBC060E9862E0A
:1041400060E0962E04C05BE8852E50E0952EE114C9
:10415000F10409F4AEC077FE06C070946194710852
:1041600073944618570817FF05C0109501951F4F07
:10417000A01AB10AD40112968C911297682F772752
:1041800067FD70958C91AB01480F511D9A01F701A5
:1041900007C08A3011F4240F351F37FD8AC03196CD
:1041A00080818823B1F7261B370BB0E820303B070E
:1041B00009F47FC0E92FF0E091FD10C093FF05C026
:1041C000A00EB11EA21AB30A09C0C801821B930B2C
:1041D00062E070E00E94EC38A60EB71EFA82E98217
:1041E0009F01217030703C832B83CF0184709070CD
:1041F0009E838D831301240C351CC401BE016F5FA7
:104200007F4F0E94F31DA0E880309A07D1F1EB8127
:10421000FC81EF2B11F062012EC02D813E81232BFA
:1042200021F06101C81AD90A26C0D301A81BB90B15
:10423000CD0162E070E00E94EC386B01C40CD51C2B
:104240001AC0D4011396ED91FC91149709958C0135
:10425000C601B501A8010E946C1CF4018181992757
:1042600087FD9095D8012C91820F911DC80ED91E03
:104270000894E11CF11CF7018081882311F08A3039
:1042800001F7D4012C9112969C91E981FA818081E9
:10429000882379F0892F992787FD9095820F911DAA
:1042A000A80EB91E7F010894E11CF11CFA82E98274
:1042B000A4CF26960FB6F894DEBF0FBECDBFCF9128
:1042C000DF911F910F91FF90EF90DF90CF90BF9003
:1042D000AF909F908F907F906F905F904F903F90A6
:1042E0002F90089582E592E00E94EA1008950E94BE
:1042F0000F120E94963704C00E9453320E941F136F
:104300000E9469128823C1F70E94AD230E94711296
:10431000089521E0FC012383089520E0FC018181C0
:1043200092818050904809F021E0822F0895CF9328
:10433000DF93EC0189819A818050904819F420E044
:1043400030E81EC08B818823C9F48881882319F046
:104350000E94741002C00E947F109C018C819D817C
:10436000281B390B89819A812817390728F4AC0159
:10437000421B530B9A0104C081E08B8320E030E0A4
:10438000C901DF91CF9108950E94972120E0892BE8
:1043900009F421E0822F0895CF93DF93EC0120E010
:1043A00089819A81892B09F421E02B8388818823D4
:1043B00019F00E94741002C00E947F109D838C83AC
:1043C000DF91CF910895CF93DF93EC010E94C42138
:1043D000882321F0CE010E94CC2181E0DF91CF9192
:1043E0000895FC01CB0125E76133720710F080E0EE
:1043F00090E892838183CF010E94CC21089560E0F0
:1044000070E80E94F1210895CF93DF93EC010E94A0
:10441000C421882321F0CE010E94FF2181E0DF9199
:10442000CF910895EEEBF6E02FEF3FEF808190E023
:104430002827392748E020FD03C080E090E002C033
:1044400088E094E83695279528273927415099F731
:10445000319686E0E73DF80749F7C9010895DF93F3
:10446000CF930F92CDB7DEB7609155067091560687
:104470006115710531F48FEF9FEF9093540680938F
:104480005306FB01E254F94F80818983282F30E0E5
:1044900080915306909154062827392748E020FD43
:1044A00003C080E090E002C088E094E8369527954C
:1044B00028273927415099F7309354062093530603
:1044C00080915206882349F0CB010496BE016F5FAC
:1044D0007F4F41E050E00E949315809155069091E6
:1044E000560601969093560680935506499710F408
:1044F00040E027C010925606109255068091520651
:10450000882381F080915306909154069093580629
:10451000809357068DE190E067E576E042E050E059
:104520000E94931540E020915306309154068091EB
:104530005706909158062817390709F041E0409333
:104540005206842F0F90CF91DF91089584E090E080
:104550006EEB76E049E150E00E9493150E94122232
:1045600090935806809357068DE190E067E576E0DA
:1045700042E050E00E9493150895AEEBB6E0EEEAFB
:10458000F1E089E101900D928150E1F70E94A622AD
:1045900008950F931F9384E090E06EEB76E049E17D
:1045A00050E00E94A1158DE190E067E576E042E0E1
:1045B00050E00E94A11500915706109158060E94E4
:1045C00012220817190711F00E94BD221F910F91A6
:1045D00008958BE596E0089510925A0610925906B8
:1045E00010925B0608952091590630915A062A359B
:1045F00031056CF4F901E55AF94F8083F9013196E0
:10460000F0935A06E0935906E55AF94F108208953F
:10461000DC010097C9F08091590690915A060DC0AF
:104620008A3591054CF4FC01E55AF94F2083019637
:10463000FC01E55AF94F108211962C91222381F743
:1046400090935A068093590608959C010097D9F0DB
:104650008091590690915A06F9014491442379F0CA
:104660008A3591054CF4FC01E55AF94F40830196D7
:10467000FC01E55AF94F10822F5F3F4FEDCF909329
:104680005A06809359060895EF92FF920F931F9355
:10469000CF93DF93AC0180E84030580729F480E6DF
:1046A00090E00E94082352C057FF18C0209159067D
:1046B00030915A062A35310574F4F901E55AF94F5B
:1046C0008DE28083F9013196F0935A06E093590602
:1046D000E55AF94F1082509541955F4F7A0100914C
:1046E000590610915A0640E0C0E1D7E201C041E00E
:1046F000C701BE010E94D838CB016AE070E00E9479
:10470000D8389C01442311F4009781F00A35110533
:1047100064F4F801E55AF94F822F805D80830F5FC2
:104720001F4FF801E55AF94F108241E0CE016AE0CF
:1047300070E00E94D838EB0161307105C1F261155B
:104740007105B1F610935A0600935906DF91CF9187
:104750001F910F91FF90EF9008950E94A622089557
:10476000009769F480EF90E00E948D21882361F129
:1047700080EF90E060E777E10E94F1210895DC018D
:1047800080E090E0282F3C91332351F0FC01EA5661
:10479000FF4F30832F5F019611968935910591F770
:1047A000E22FF0E0EA56FF4F108280EF90E060E7E2
:1047B00077E10E94F12180E090E89093F7008093E8
:1047C000F60081E08093F8000895FC01A6E9B0E0CE
:1047D00080E09491992329F09D938F5F31968935DC
:1047E000C1F7E82FF0E0EA56FF4F108286E990E02B
:1047F0000E94B0230895809195008150823010F17D
:1048000081E00E9493118823E9F083E00E949311D4
:104810000E940212882349F080E00E94051283E082
:104820000E945B118EE795E108C081E00E940512AD
:1048300082E00E945B1184E795E10E94E52381E01C
:104840008093F80008950F931F93CF93DF938AEF1F
:1048500090E00E94E321882309F441C00E940212E3
:104860008823C9F00E943211282F30E08091F9008E
:10487000882341F0E9012196C436D1056CF11092EC
:10488000F9002AC0E9012197C531D1052CF581E055
:104890008093F90021C00E943211C82FDD27C7FD87
:1048A000D09580919500882319F000E010E00CC0AD
:1048B0000E9435118C018431910524F00E949310DF
:1048C000882311F404E110E0C017D1070CF42196FD
:1048D0000C171D070CF421978C2F0E941411DF91E7
:1048E000CF911F910F91089590E0FC013197EA312B
:1048F000F10508F056C0EB59FF4FEE0FFF1F059072
:10490000F491E02D09948CE898E14DC081E898E19C
:104910004AC084E798E147C088E698E144C08EE544
:1049200098E141C081E598E13EC083E498E13BC055
:1049300088E398E138C08BE298E135C08FE198E1D7
:1049400032C083E198E12FC082E098E12CC083EF70
:1049500097E129C085EE97E126C088ED97E123C055
:1049600089EC97E120C08AEB97E11DC08BEA97E1C3
:104970001AC08DE997E117C082E997E114C089E870
:1049800097E111C08DE797E10EC08DE697E10BC06E
:104990008DE597E108C083E597E105C088E497E1DC
:1049A00002C080E497E10E94252308950F931F938E
:1049B0008C010E943F1181E090E061E0A8010E941B
:1049C0004C1A1F910F910895BF92CF92DF92EF92F0
:1049D000FF920F931F93DF93CF9300D000D0CDB7FA
:1049E000DEB77C01FC01828193818859984008F0F0
:1049F00032C1C7010E9488198C0120E880309207DB
:104A000011F490E030C1F701C280D380C6018C560A
:104A1000974063E170E00E94D838B82E2C2D2370A7
:104A2000C6018956974067E070E00E94D83830E0B0
:104A3000E82FF0E084E3C81688E0D806A8F483E104
:104A4000B89EC001112448966EE170E00E94EC38D7
:104A5000482F220F331FEE0FFF1FEE0FFF1F2E0FE9
:104A60003F1F2B5F3F4F14C083E1B89EC00111244C
:104A700048966EE170E00E94EC38482F220F331FF9
:104A8000EE0FFF1FEE0FFF1F2E0F3F1F2A5F3F4F3E
:104A900086E0489FC0011124820F931F67E070E0F9
:104AA0000E94EC38282F842F90E0820F911D240F54
:104AB0000A9724F42A5E298383E011C0822F89504B
:104AC00089838A3111F483E108C0893139F44C318A
:104AD00029F4EAE0EB1510F482E1898384E08A830B
:104AE000DC82CB82CE0101960E948819D82E88E103
:104AF00089838CE08A83F701828193819C838B83F5
:104B0000CE0101960E944B19873011F456E102C084
:104B100056E1581BF7014181413049F480818130D1
:104B200011F492E0A0C0863011F493E09CC02D2DCA
:104B300030E0C901C4978017910711F494E093C045
:104B4000C901C0978017910711F495E08CC0C90185
:104B50008F978017910711F496E085C0C9018E9751
:104B60008017910711F497E07EC0C9010397801761
:104B7000910711F498E077C0C90102978017910757
:104B800011F499E070C02017310711F49AE06BC05E
:104B9000C90101968017910711F49BE064C045306C
:104BA00031F4F7018081813011F49CE05CC0C901CF
:104BB00087968017910711F49DE055C0C901C196F1
:104BC0008017910711F49EE04EC0C901C29680176C
:104BD000910711F49FE047C0245C3F4F2017310735
:104BE00011F490E140C0483031F4F70180818F30FA
:104BF00091F591E138C04A3051F4F701808183305A
:104C000011F492E130C08F3131F593E12CC04B307B
:104C100051F4F7018081813011F494E124C08517AB
:104C2000D1F495E120C04C30B1F4F7018081863099
:104C300011F496E118C0883111F497E114C089315C
:104C400011F498E110C08A3111F499E10CC08F3150
:104C500011F49AE108C0C7010E944B1990E08650F8
:104C6000823008F491E0892F0F900F900F900F90F1
:104C7000CF91DF911F910F91FF90EF90DF90CF9038
:104C8000BF9008951F93182FCB010E94E424282F72
:104C90008230E8F0E5E3F7E184912817B1F031962E
:104CA00087E1E034F807C1F7E12FF0E0EE0FFF1FD6
:104CB000EE0FFF1FEB50F94E90E08491281729F07A
:104CC0009F5F31969430C9F702C081E001C080E057
:104CD0001F9108951F93CF93DF93EC010E94421719
:104CE000882391F0888190E00E9444238AE30E9407
:104CF000F32219811A3018F480E30E94F322812FE5
:104D000090E00E94442304C084EA98E10E94252395
:104D1000DF91CF911F910895EF92FF920F931F9310
:104D2000DF93CF93CDB7DEB72E970FB6F894DEBFE3
:104D30000FBECDBF8E010F5F1F4FC8010E94D6244A
:104D40008091C506882309F46FC0C8010E94AF197D
:104D5000882309F469C0DE011896E7ECF6E087E0E5
:104D600001900D928150E1F781E090E061E0AE01A9
:104D7000485F5F4F0E944C1A8E010C5F1F4FBBE0D3
:104D8000EB2EF12CEC0EFD1EC801B7010E94E617B8
:104D9000882319F48FEE96E139C0C8010E942F19BB
:104DA000C801B7010E94E617882319F488EE96E13E
:104DB0002DC0C8010E942F19C801B7010E94E61733
:104DC000882319F48DED96E121C08091D606B701B4
:104DD0000E944226882331F0C7010E94E4240E94E9
:104DE000742416C083ED96E10E942523C7010E941A
:104DF0004B19982F8150873008F090E0E92FF0E0B0
:104E0000EE0FFF1FEC56F74E859194910E942523DB
:104E100080ED96E10E942523CE0108960E946A2625
:104E20008AEC96E10E9425232E960FB6F894DEBFF9
:104E30000FBECDBFCF91DF911F910F91FF90EF90EB
:104E40000895CF92DF92EF92FF920F931F93E82E77
:104E50008B016A010E94EC22C8010E944423C60112
:104E60000E9425230E94E9226C01FF24E7FCF094B4
:104E700080E060E070E0A7012FE730E000E110E0A3
:104E800094E0E92E0E947D201F910F91FF90EF90FA
:104E9000DF90CF900895CF92DF92EF920F931F9300
:104EA000E82E8A0108C0F80184910F5F1F4F8C32F1
:104EB000D1F76150704016161706ACF30E94EC2231
:104EC000F8018491882339F08C3229F00E94F32272
:104ED0000F5F1F4FF5CF0E94E9226C014E2D552721
:104EE00047FD509580E06FE770E020E030E000E1A2
:104EF00010E0E4E0EE2E0E947D201F910F91EF90D4
:104F0000DF90CF9008952F923F924F925F926F92D1
:104F10007F928F929F92AF92BF92CF92DF92EF9249
:104F2000FF920F931F93DF93CF93CDB7DEB72C97EC
:104F30000FB6F894DEBF0FBECDBF9C878B874B01A9
:104F40006A0119012801FE2C0E94EC22C8010E946E
:104F50006A266624772410E005E0A02EB12CAC0E62
:104F6000BD1E0E94E922212F30E0FC01E20FF31F59
:104F70008081F501E20FF31F80838A3311F41192CF
:104F80003F011F5F0E94E922FC01E10FF11D3197F3
:104F90008081882331F7C60162E070E00E94EC381E
:104FA0005B018B859C85A80EB91EF20180818A3039
:104FB00050F4FF2019F086EF9FEF09C0EAEFFFEFF2
:104FC000AE0EBF1E06C0FF2021F088EF9FEFA80E97
:104FD000B91EB5016750704081E0A40120E030E0C7
:104FE0008101B4E0EB2EA5E0CA2ED12CCC0EDD1E43
:104FF0000E947D2081E0B501A40120E030E0EE2494
:10500000F4E6CF2EF0E0DF2E0E947D20E7E0F0E016
:10501000AE0EBF1E81E0B501A40120E030E0EE2419
:10502000E39463010E947D20FF2009F441C081E0E8
:10503000B301AE014F5F5F4F9E012D5F3F4F0E9456
:105040000D2009811A810E94EC22C2010E944217A0
:10505000882369F0F201E280F9E0FE1518F080E3A0
:105060000E94F3228E2D90E00E94442304C08AEA1D
:1050700098E10E9425230E94E9226C0182E090E0E1
:10508000880E991E0D5F1F4F0A0D1B1DC10162E0A6
:1050900070E00E94EC38860E971E80E0B801A401F3
:1050A00020E030E00DE010E0EE24E3940E947D204B
:1050B0002C960FB6F894DEBF0FBECDBFCF91DF9117
:1050C0001F910F91FF90EF90DF90CF90BF90AF9026
:1050D0009F908F907F906F905F904F903F902F9018
:1050E00008950F931F93DF93CF9300D0CDB7DEB712
:1050F0008C010E94B02380EF90E00E94FF2180E0AD
:10510000B80148EB56E09E012F5F3F4F0E940D20F3
:10511000882391F085E890E09093F7008093F60063
:1051200080EB9FEF2091B8063091B906821B930B5C
:105130009093B9068093B8060F900F90CF91DF91AE
:105140001F910F9108950E94E52386E990E00E9447
:1051500071280895DF92EF92FF920F931F93DF93D0
:10516000CF93CDB7DEB72E970FB6F894DEBF0FBE44
:10517000CDBFD82EDE011196E7ECF6E087E0019076
:105180000D928150E1F781E090E061E07E010894AA
:10519000E11CF11CA7010E944C1A8E01085F1F4FF1
:1051A000C8010E94D624C8010E94AF19882309F4BF
:1051B0006DC08B859C85AD85BE858C839D83AE83BC
:1051C000BF83C701B8010E94BE17181624F0CE0194
:1051D00004960E942F1984E0E82EF12CEC0EFD1E9F
:1051E00001E0C7010E944B1910E08650823008F49C
:1051F00011E08091D606B7010E94422693E0D916AD
:10520000E1F09D1538F091E0D91659F092E0D916E9
:1052100059F509C094E0D91699F095E0D91621F511
:105220001AC0812F1BC0112321F420E030E0882315
:1052300011F021E030E0822F11C01123A9F410C039
:10524000112319F080E090E009C090E0811191E015
:105250009027892F03C0882339F402C0882321F0C6
:10526000C7010E942F19BDCFA7ECB6E0FE01319611
:1052700087E001900D928150E1F71092C90681E01C
:1052800090E061E047EC56E00E94A91A2E960FB616
:10529000F894DEBF0FBECDBFCF91DF911F910F916C
:1052A000FF90EF90DF900895DF92EF92FF920F93BF
:1052B0001F93DF93CF93CDB7DEB72A970FB6F8943D
:1052C000DEBF0FBECDBF8FE191E00E94E3218823B6
:1052D00071F0CE0104960E943F119E818091BA0622
:1052E000891719F081E08093F8009093BA068091B5
:1052F000B706882309F450C0CE0101960E948A1097
:1053000000E08A819B818D57914008F001E0D090A8
:10531000C0060E940212182F8091C506882321F032
:1053200080919500833071F480E091E00E94C42167
:10533000882341F01123C1F40023B1F440E8E42EA6
:10534000F12C16C0112309F40111DD24002341F4CE
:10535000112331F4DD2021F03AE7E32EF12C08C0CF
:105360002AE6E22EF12C04C09AE6E92EF12CDD2487
:105370008E010C5F1F4FC8010E94D62480E090E090
:1053800060E070E0A7012FE230E0ED2C0E9483275F
:105390008FE191E00E94CC212A960FB6F894DEBFEF
:1053A0000FBECDBFCF91DF911F910F91FF90EF9076
:1053B000DF900895DF93CF9300D00F92CDB7DEB783
:1053C00089E191E00E94E321882339F1CE01019621
:1053D0000E948A108A819B81039718F00E94921282
:1053E00002C00E94FE148823C1F480EF90E00E9466
:1053F0008D21882391F420E08091F6009091F700B0
:105400008050904809F021E0222339F48FE00E9477
:105410005B118AED98E10E94E5230F900F900F90A9
:10542000CF91DF910895CF92DF92EF920F931F9368
:10543000DF93CF93CDB7DEB727970FB6F894DEBFD3
:105440000FBECDBF80EF90E00E948D21882361F0D8
:1054500011E01093180180EF90E00E94042288234D
:1054600099F11093F80030C08091F6009091F70008
:105470008050904801F181E08093180181E491E02F
:105480000E94E321882301F18091F6009091F700BA
:1054900001979093F7008093F6002091B806309121
:1054A000B9068217930769F480E090E89093F700BB
:1054B0008093F60006C08BE391E00E94C42188230C
:1054C00019F081E08093F8008091B706882309F4F1
:1054D000DAC080E090E06FE270E040E850E021E068
:1054E00030E00E94FF1E80EF90E00E948D21882313
:1054F00061F080E060E070E04FE250E020E830E0F2
:1055000001E110E0F8E0EF2E11C06091F60070911B
:10551000F70080E86030780781F080E04FE250E0EB
:1055200020E137E201E110E0E9E0EE2E96E9C92E34
:1055300090E0D92E0E947D20A6C0CE0101960E9447
:10554000D624CE0104960E94E424182F0E94EC2257
:105550008091D506882329F0112319F0113009F024
:1055600045C08E010C5F1F4FC8010E94651888233B
:1055700009F437C0C8010E944B19880F8250082FC8
:1055800010E0F801EE5CF64EE4918E2F0E94F322BB
:105590000D5C164EF80184910E94F3228EEF98E183
:1055A0000E9425238C8190E00E9444238BEF98E198
:1055B0000E94252300E010E0ED81F0E03197EE0F2E
:1055C000FF1FEE0FFF1FE00FF11FEF5FF64EE4919C
:1055D0008E2F0E94F3220F5F1F4F0430110561F7D9
:1055E00008C08EEE98E10E94252303C0812F0E94FF
:1055F00074248091D406882319F4A8E0EA2E02C00E
:10560000F9E0EF2E0E94E9226C0180E060E070E09A
:105610004FE250E020E830E001E110E00E947D2000
:105620008091D406882359F10E943A1190933A014F
:10563000809339010E94EC228091390190913A01C6
:10564000F0E880309F0729F48AEE98E10E94252334
:1056500002C00E94442387EE98E10E9425230E9405
:10566000E9226C0180E060E070E04FE250E020E869
:1056700030E001E110E0ECE0EE2E0E947D208BE3B3
:1056800091E00E94CC2127960FB6F894DEBF0FBEA2
:10569000CDBFCF91DF911F910F91EF90DF90CF9011
:1056A00008951F9380E00E94F511182F8091BC0689
:1056B000811749F480E00E949311882321F40E940D
:1056C000C411882329F01093BC0681E0809318014F
:1056D00080911801882399F01092180187E491E0D5
:1056E0000E948D21882319F481E00E94B9106091F5
:1056F000BE067091BF0687E491E00E94F12187E425
:1057000091E00E940422882319F080E00E94B910E1
:105710008091B706882331F01092B7060E9472215B
:105720000E94371E8091F800882329F01092F8001B
:1057300081E08093B7061F9108952F923F924F9278
:105740005F926F927F928F929F92AF92BF92CF9211
:10575000DF92EF92FF920F931F93DF93CF93CDB71A
:10576000DEB761970FB6F894DEBF0FBECDBF9C8742
:105770008B874B011A0129011E870D873701DE0136
:105780001596E6E0F2E086E001900D928150E1F797
:10579000ED85FE85C080D18081E08093F8008E0188
:1057A0000B5F1F4FC8010E94CC21098BF12EC40151
:1057B0000197988B8F87B7C081E00E94C41188231E
:1057C00031F083E00E94C4118DE00E945B11898951
:1057D0009F2D0E94C421882321F08EE00E945B113E
:1057E000A8C081E00E94F511182F882311F45601FA
:1057F00033C081E00E94F511212F332727FD30951A
:1058000094E6C916D10424F4C9018C0D9D1D0EC067
:10581000C60165E070E00E94EC38620F731FCB0197
:10582000880F991F880F991F860F971F48165906D2
:105830000CF4C2015C01821593050CF45101CA14E9
:10584000DB0419F081E00E945B1189899F2D0E9481
:10585000CC2181E08093F8008091B706882309F479
:1058600056C00E94EC228B859C850E9425230E94B5
:10587000E9226C0180E06DE070E0A40120E830E0F6
:105880000FE010E0EE24E3940E947D2083E160E0CD
:1058900070E0A4012BE030E000E110E00E94B11FB5
:1058A0000E94E922BC0180E0AE014F5F5F4F9E0184
:1058B0002D5F3F4F0E940D2089819A810E969A8319
:1058C000898340E850E0481B590B6F85788921E1B6
:1058D00030E00E94FF1E0E94EC22C5010E9444237A
:1058E0006114710419F0C3010E94252309811A81F2
:1058F0000E94E9226C0120E830E0201B310B80E09F
:10590000B801A4010FE010E0EE240E947D200E9467
:10591000FB230E94512B0E94232481E080931801D5
:105920000E941F13650182E00E94C411882309F4BC
:1059300043CF82E00E94C411882321F0ED85FE85CB
:10594000D182C08283E00E94C41181E08093F8007C
:1059500061960FB6F894DEBF0FBECDBFCF91DF9139
:105960001F910F91FF90EF90DF90CF90BF90AF907D
:105970009F908F907F906F905F904F903F902F906F
:1059800008959F92AF92BF92CF92DF92EF92FF92D3
:105990000F931F93DF93CF9300D000D000D0CDB7EB
:1059A000DEB75C01DE011196ECE0F2E086E00190EA
:1059B0000D928150E1F781E08093F8008E010F5F36
:1059C0001F4FC8010E94CC21902EF12E32C0809131
:1059D000B706882341F188E090E062E070E048E794
:1059E00050E02CE330E00E94FF1E89E090E063E08D
:1059F00070E046E750E02AE330E00E94FF1E0E947C
:105A0000EC22C5010E9425230E94E9226C0180E05E
:105A100069E070E043E050E026E730E00AE310E0A0
:105A2000EE240E947D200E94512B0E9423240E947C
:105A30001F1381E00E94C411882359F40E94F511BC
:105A4000882339F4892D9F2D0E94C421882309F4CD
:105A5000BECF83E00E94C41181E00E94F51181E075
:105A60008093F80026960FB6F894DEBF0FBECDBF28
:105A7000CF91DF911F910F91FF90EF90DF90CF902A
:105A8000BF90AF909F9008950F931F9300914D0189
:105A900010914E010E9435110817190741F00E941C
:105AA000351180934D0190934E010E9496108FE422
:105AB00091E00E94E321882321F10E940C12609161
:105AC000BD068823C9F0862F90E02091C106309151
:105AD000C206A90113E0440F551F1A95E1F7220FE2
:105AE000331F420F531F8417950714F46F5F07C0CD
:105AF00081E08093180105C0662319F0615060931E
:105B0000BD061F910F9108957F928F929F92AF9241
:105B1000BF92CF92DF92EF92FF920F931F93DF938A
:105B2000CF9300D000D000D0CDB7DEB74C01DE015E
:105B30001196E2E1F2E086E001900D928150E1F7EA
:105B400081E08093F8008E010F5F1F4FC8010E9413
:105B5000CC217724FF245801ADC080E00E94F511CC
:105B6000182F882381F081E00E945B1181E00E9460
:105B7000F511F12EFF1CFF24FF1C81E08093F8003B
:105B8000C5010E94CC2181E00E94C411882359F0F4
:105B900083E00E94C41181E08093F800C5010E9457
:105BA000CC21772473948091B706882309F479C0B7
:105BB00084E090E062E070E048E750E02CE330E001
:105BC0000E94FF1E85E090E063E070E046E750E051
:105BD0002AE330E00E94FF1E0E94EC22C4010E94D2
:105BE00025230E94E9226C0180E068E070E045E036
:105BF00050E020E730E001E210E093E0E92E0E945F
:105C00007D2088E090E069E270E047E350E021E128
:105C100030E00E94FF1E0E94EC2283E59CE10E947E
:105C200025230E94E9226C0180E068E070E049E2EF
:105C300050E027E330E001E110E0EE240E947D20F7
:105C400081E490E069E270E046E350E021E130E079
:105C50000E94FF1E0E94EC228EE49CE10E942523FC
:105C60000E94E9226C0180E061E470E049E250E0CA
:105C700026E330E00E947D20772099F4FF2039F060
:105C80008AE090E06BE270E043E350E006C083E41A
:105C900090E06BE270E042E350E02DE030E00E94E3
:105CA000BF1E0E94512B0E94232481E08093180183
:105CB0000E941F1382E00E94C411882331F4C501A1
:105CC0000E94C421882309F448CF8DE00E945B1113
:105CD00083E00E94C41181E00E94F51181E080936D
:105CE000F800CE0101960E94C4218111FF248F2D5E
:105CF00026960FB6F894DEBF0FBECDBFCF91DF91D1
:105D00001F910F91FF90EF90DF90CF90BF90AF90D9
:105D10009F908F907F9008952F923F924F925F9225
:105D20006F927F928F929F92AF92BF92CF92DF92AB
:105D3000EF92FF920F931F93DF93CF93CDB7DEB710
:105D400027970FB6F894DEBF0FBECDBF80919500A8
:105D5000833019F0882309F089C380E00E94C411C0
:105D6000882309F483C385E591E00E94C421882338
:105D700009F480C3DE011196E0E0F2E086E00190D4
:105D80000D928150E1F78CE00E945B11BB24AA24A4
:105D9000A39498E2892E912CA092F8008091B706E6
:105DA000882309F443C080E060E070E040E050E008
:105DB00020E830E00CE210E0EE240E94B11F0E94C7
:105DC000EC2282E29CE10E9425230E94E9226C01E0
:105DD00080E060E070E04FE250E020E830E001E178
:105DE00010E00E947D2080E090E06FE270E040E8EB
:105DF00050E021E130E00E94BF1E0B2D10E0740145
:105E0000E01AF10A80E090E060E070E0A7012FE284
:105E100030E00E947F1EC801885A9F4F60E070E00A
:105E2000A7012FE230E00E947F1EB3940E94FB2363
:105E30000E9423240E94512B0E941F1387E28B157E
:105E400008F0AACF0E94371E83E00E94C41181E0AF
:105E50000E94F5118E010F5F1F4FC80160E27EE4C2
:105E60000E94F12181E08093F800A12C80E8B82EF7
:105E7000FF2433240F83212ED9C28F81922D0E94BB
:105E8000C421882321F08EE00E945B11D6C281E0FC
:105E90000E94F511482F882311F46F2C27C06F2C16
:105EA0000EC09DE0961508F06394262D30E0832DFA
:105EB00090E00396821793070CF433944150141624
:105EC00084F306C061106A94631408F43A944F5F37
:105ED0004423C1F78F81922D0E94CC21F61431F01A
:105EE00081E00E945B1181E08093F80081E00E94D4
:105EF000C411882309F449C083E00E94C4118DE0D5
:105F00000E945B1182E0681609F1861530F0662068
:105F100059F091E06916A1F510C084E06816F9F017
:105F20009BE0691669F524C090E08091C006882343
:105F300009F491E09093C00623C090E08091D406CC
:105F4000882309F491E09093D4061AC090E08091E0
:105F5000CE06882309F491E09093CE0611C090E01C
:105F60008091D106882309F491E09093D10608C06E
:105F700090E08091D506882309F491E09093D506AE
:105F8000A62CBB2481E08093F80082E00E94C4111B
:105F9000882309F456C183E00E94C411862D90E045
:105FA000A816B90609F043C1F501EE0FFF1FE05D29
:105FB000F34E25913491C50183199109682F62959B
:105FC000607F88E0A816B10409F475C099E0A916AD
:105FD000B104D4F485E0A816B10409F443C096E0F6
:105FE000A916B10434F483E0A816B10409F01FC166
:105FF0002AC096E0A916B10409F445C087E0A816A6
:10600000B10409F014C14AC09CE0A916B10409F416
:10601000F3C08DE0A816B1045CF499E0A916B104B0
:1060200009F458C08AE0A816B10409F000C184C080
:106030009DE0A916B10409F4ECC08EE0A816B104E5
:1060400009F0F5C0F0C0772767FD7095C90143E0FE
:1060500050E020EE31E00FEC16E0AEE1EA2EACE1CC
:10606000FA2E0EC0772767FD7095C90142E050E017
:106070002AE530E002ED16E0FAE1EF2EFCE1FF2E1A
:106080000E949D2BD4C0772767FD7095C90141E020
:1060900050E029E030E003EC16E00AC0772767FD06
:1060A0007095C90141E050E029E030E001EC16E0D4
:1060B000EE24FF24E5CF772767FD7095C90145E001
:1060C00050E027EE33E00EEB16E0E8E1EE2EECE1D7
:1060D000FE2ED6CF8091C6068F5F8093C60687308E
:1060E00010F01092C6068091C6068230B1F083305F
:1060F00028F4882351F08130E1F40AC0843099F00B
:10610000843070F08530A9F411C08CE09CE102C0AD
:1061100083EE9BE10E94C12C8AC083EB9BE1FACF06
:106120008CE99BE1F7CF85E79BE1F4CF8FE59BE11D
:10613000F1CF8DE39BE1EECF8091D6068F5F809308
:10614000D606803110F01092D6068091D6068730A0
:10615000C1F1883070F4833041F1843028F481300B
:10616000F1F08230F8F418C0853029F1863030F52E
:106170001FC08B3091F18C3028F4893041F18A3086
:1061800048F522C08D3079F18D3050F18E3071F1AB
:106190008F3009F04CC02DC085E29BE1BBCF89E177
:1061A0009BE1B8CF8DE09BE1B5CF8CEF9AE1B2CF08
:1061B00080EF9AE1AFCF83EE9AE1ACCF87ED9AE121
:1061C000A9CF8AEB9AE1A6CF87EA9AE1A3CF8DE81F
:1061D0009AE1A0CF88E79AE19DCF8AE69AE19ACF2B
:1061E0008DE59AE197CF89E49AE194CF81E39AE132
:1061F00091CF82E29AE18ECF80E09AE10E94842DD5
:106200008823A9F083E991E00E944D110E94FE14B9
:1062100008C08DED99E10E94842D882341F00E94F1
:10622000BD220E9470108F81922D0E94FF218F81CC
:10623000922D0E94CC2181E08093F800A12CB0E83F
:10624000BB2E8091B706882309F4E4C0F32C882480
:106250009924DBC00E94EC22EF2DF0E0EE0FFF1F2F
:10626000E05DF34E859194910E942523582C492C92
:106270000E94E9226C0180E06DE070E0A40121E75A
:1062800030E00FE010E0EE24E3940E947D20F6144D
:1062900049F483E160E070E0A4012BE030E000E12C
:1062A00010E00CC0A4014B5F5F4F84E163E070E03D
:1062B00025E030E005E010E0EE24E3940E94B11FF9
:1062C00095E0F91609F447C09F15A0F082E0F81692
:1062D00081F18F1538F0FF2031F191E0F91609F0C6
:1062E0007CC024C083E0F81659F194E0F91609F057
:1062F00074C02EC088E0F81609F444C08F1540F031
:1063000096E0F91691F187E0F81609F066C032C000
:106310009AE0F91609F445C0F916E0F18BE0F81699
:1063200009F05BC047C08091C00646C08091D4068A
:1063300043C06091CE06872D70E040ED59E137C033
:106340006091CF067091D006872D4CEC59E10AC0C0
:106350008091D10631C06091D2067091D306872D0D
:1063600048EC59E10E94212738C06091C306709122
:10637000C40604C06091C1067091C206872D40E03A
:1063800050E0F0CF6091BE067091BF06872D46ECBD
:1063900059E1E8CF6091C606872D70E043EB59E1E3
:1063A00006C06091D606872D70E043E859E10E944F
:1063B0004B2713C08091D506882311F486E101C0D4
:1063C00085E160E070E0452D542D2FE730E000E1DD
:1063D00010E0E4E0EE2E0E94B11F8F2D90E08A15B0
:1063E0009B0551F48CE090E0652D742D44E750E05E
:1063F00020E130E00E94BF1E80E190E0880E991EEF
:1064000090E48916910431F0F394782C8EE08F1586
:1064100008F020CF0E94FB230E9423240E94512BCE
:1064200081E0809318010E941F13F62C8F81922D1A
:106430000E948D21882309F020CDCE0101960E9473
:10644000C421882319F087E599E102C081E499E12C
:106450000E94A32882E191E062E070E00E94F121B5
:1064600083E00E94C41181E00E94F51185E591E06E
:106470000E94CC2127960FB6F894DEBF0FBECDBF89
:10648000CF91DF911F910F91FF90EF90DF90CF9010
:10649000BF90AF909F908F907F906F905F904F9044
:1064A0003F902F9008953F924F925F926F927F920C
:1064B0008F929F92AF92BF92CF92DF92EF92FF9214
:1064C0000F931F93DF93CF93CDB7DEB7A4970FB68B
:1064D000F894DEBF0FBECDBF0E94FB230E94232491
:1064E00080919500813009F4F1C181E00E94F5119D
:1064F000882309F4EBC1DE011496E7EDF1E086E0B4
:1065000001900D928150E1F7DE011A96E1EDF1E084
:1065100086E001900D928150E1F784E00E945B11CA
:106520008BEB96E10E94E523DE015E96E7ECF6E058
:1065300087E001900D928150E1F78E01025E1F4FBE
:1065400081E090E061E0A8010E944C1A2F8D822F1B
:1065500065E00E94CC38291B2F8F6DE7C62ED12C09
:10656000B02EF12E0E9454290E94132A8091B70662
:10657000882309F43FC0C6010396079748F0C60177
:1065800064E070E00E94EC38C61AD70AD7FE02C059
:10659000CC24DD24C601039760E070E041E050E0C8
:1065A0002FE230E00E943F1EC601029760E070E0DB
:1065B00040E850E02FE230E00E947F1EC601429684
:1065C00060E070E04EE650E02FE230E00B2D1F2D32
:1065D000EE240E94832787E0B60140E050E020E8E7
:1065E00030E00EE210E0EE24E3940E94B11F81E05F
:1065F0008093F8000E9423240E94512B0E941F13B5
:106600001C141D040CF4AECF81E00E94F51183E050
:106610000E94C4118E010C5F1F4FC8010E94CC2143
:10662000AA24B02EF12E772473945AE0452E512CD3
:106630004C0E5D1E4EE1842E912C8C0E9D1E3CE373
:10664000632E28E1322E22E130E0C20ED31EDAC0E2
:106650007092180180E090E00E94B023C2010E9475
:10666000E321882339F0A39439E03A1508F4AA24E9
:106670007092F800C4010E944217882389F181E0DA
:106680000E94F511182F882359F181E00E945B11B7
:106690000DC08F8D8B5F8F8F8C3339F41F8E8E8D55
:1066A0008F5F8E8F883109F41E8E115011168CF376
:1066B0000FC08F8D882341F48E8D882309F43E8E80
:1066C0008E8D81508E8F6F8E8F8D85508F8F1F5F37
:1066D00017FDEFCF7092F8008B2D9F2D0E94CC21DB
:1066E00081E00E94C411882359F185E00E945B116A
:1066F000A7ECB6E0F40187E001900D928150E1F73C
:106700001092C90681E090E061E047EC56E00E94FB
:10671000A91A80E00E94AA287092C50610929500DE
:106720000E94EC2285EA96E10E9425230E948C2695
:106730000E94E9220E9471288B2D9F2D0E94FF212B
:106740008B2D9F2D0E94C421882381F1C4010E94BA
:106750004217882339F1D401E3E9F1E087E00190A1
:106760000D928150E1F78EE00E945B118091C50689
:10677000882369F00E94EC2288E696E10E94252396
:106780000E948C260E94E9220E94712804C087E39F
:1067900096E10E94A3288B2D9F2D62E070E00E945D
:1067A000F12104C08B2D9F2D0E94FF218091B706FF
:1067B0008823E1F0C60160E070E04EE650E02FE291
:1067C00030E08401EE240E948327EA2DF0E0E953B3
:1067D000FE4F808160E070E040E050E020E830E073
:1067E0000EE210E0EE24E3940E94B11F0E94132AEF
:1067F0000E94FB230E9423240E94512B0E94442DBF
:106800000E941F138B2D9F2D0E948D21882309F03C
:106810001FCF94E0C92ED12C8EE1A82EB12CAC0E46
:10682000BD1E0E9454290E94132A8091B706882316
:10683000B1F1C601039760E070E041E050E02FE263
:1068400030E00E943F1EC601029760E070E040E821
:1068500050E02FE230E00E947F1EC6010E9660E0FD
:1068600070E042E750E02FE230E08501EE240E9424
:10687000832787E0B60140E050E020E830E00EE2F8
:1068800010E0EE24E3940E94B11F81E08093F800B1
:10689000C60163E070E00E94EC38C60ED71E0E946D
:1068A00023240E94512B0E941F1381E00E94F511A6
:1068B000882329F480E8C816D1040CF4B2CF80E014
:1068C00091E00E94892183E00E94C411809195008B
:1068D000882311F0833099F581E00E94C411882348
:1068E00071F183E00E94C4118091C506882389F06C
:1068F00087E00E945B111092C50683E080939500AB
:1069000080E091E065E070E00E94F12183E296E191
:106910000EC08091C6060E94AA2881E08093C50619
:106920001092950086E00E945B1182E196E10E9440
:10693000E52382E191E062E070E00E94F121809124
:106940009500813009F48FC0813038F0823009F42D
:106950004CC1833009F0B5C17CC1DE015E96E7EC25
:10696000F6E087E001900D928150E1F70EE1C02E34
:10697000D12CCC0EDD1EC6010E94D91982E388A35A
:106980008E01095E1F4FC8010E943F11C8010E947D
:10699000AF19882349F0C801B6010E94E91987FDA3
:1069A00003C081E0809318018E01095E1F4FC8016A
:1069B0000E943F11C8010E94AF19882309F483C1C6
:1069C0008091C906898F87EC96E0B8010E94E91989
:1069D00018160CF478C188E00E945B118091C606FD
:1069E0000E94AA288091CE068823E1F40E94021218
:1069F0008823C1F080EF95E10E94A3288091C6060C
:106A0000863011F41092C50680E091E064EB70E0EE
:106A10000E94F12182E191E062E070E00E94F121A8
:106A200083E01EC08EED95E10E94E5232091CF0604
:106A30003091D0068CE390E0289FB001299F700D23
:106A4000389F700D11248CE091E00E94F12186E0C6
:106A500091E062E370E00E94F1211092B60681E0BD
:106A60008093950030C18091CE06882341F00E942A
:106A70008811882339F48AE00E945B1103C081E009
:106A80000E94051281E00E94F51181E00E94C4116C
:106A9000882359F481E00E949311882331F48CE01B
:106AA00091E00E94C421882371F181E08093180154
:106AB00089EC95E10E94A32882E191E062E070E018
:106AC0000E94F12183E00E94931183E00E94C4118F
:106AD00089E00E945B118091CE06882311F40E9408
:106AE000051280E00E9405128091C606863011F4DE
:106AF0001092C50683E08093950080E091E064EBFE
:106B000070E00E94F1218091D106882309F469C0C8
:106B100086E091E00E94E321882309F462C00E948C
:106B20000C126091B606882309F456C0862F90E0B7
:106B30002091C3063091C406A90113E0440F551FEC
:106B40001A95E1F7220F331F420F531F8417950741
:106B500014F46F5F44C08DE00E945B118091CE06FB
:106B6000882311F40E9405120E94EC228CEB95E11F
:106B70000E9425238091D2069091D3060E9444233F
:106B800081EB95E10E9425230E94E9220E94712851
:106B90008E01005F1F4FC8010E943F11C8010E9473
:106BA000AF19882309F41A8A2091D2063091D306AE
:106BB0008CE390E0289FB001299F700D389F700DE5
:106BC00011248A89681B71098CE091E00E94F121EF
:106BD00082E08093950005C0662319F061506093B0
:106BE000B60681E0809318016EC081E00E94C41156
:106BF000882361F481E00E949311882339F48CE0AA
:106C000091E00E94C421882309F45DC011E0109333
:106C100018018DE995E10E94A32886E091E062E3E6
:106C200070E00E94F1211092B6062091CF063091BB
:106C3000D0068CE390E0289FB001299F700D389F0B
:106C4000700D11248CE091E00E94F12110939500C9
:106C50003AC08091C5068823B1F1DE015796E7EC72
:106C6000F6E087E001900D928150E1F78F898A303C
:106C700038F4825F8F8BCE014A960E94EF1802C0D3
:106C80008A508F8B8E01025E1F4FC8010E943F11F8
:106C900088A1898FC8010E94AF198823A1F0C8017B
:106CA000BE01695E7F4F0E94E91987FD0CC081E03B
:106CB0008093180188E895E10E94A3288BE00E9448
:106CC0005B111092950080EF90E00E948D21882347
:106CD00039F520E08091F6009091F70080509048BF
:106CE00009F021E02223E1F482E191E00E940422F4
:106CF000882311F18091C506882369F00E94EC2257
:106D000084EC98E10E9425230E948C260E94E922AF
:106D10000E94712811C08DEA98E10E94A3280CC03E
:106D200082E191E00E948D21882331F082E191E09F
:106D300062E070E00E94F1210E94DA290E94542949
:106D4000809195008130C1F485E291E00E94C421D8
:106D5000882391F085E291E062E370E00E94F121E6
:106D60008091BB068F5F8093BB068A3010F0109233
:106D7000BB0681E08093F800809195008230C1F4D9
:106D800085E291E00E94C421882391F085E291E0A0
:106D900064E670E00E94F1218091BB068F5F8093D2
:106DA000BB06893110F01092BB0681E08093F80099
:106DB0008091B7068823A1F180919500813031F050
:106DC000813008F4B1C0823071F406C0E091BB0696
:106DD000F0E0EA50FE4F05C0E091BB06F0E0E35260
:106DE000FE4F808111C0833071F480E091E00E94F9
:106DF0008D21882341F080E091E00E94C421882306
:106E000011F489E001C089E260E070E040E050E008
:106E100020E830E00EE210E0A6E0EA2E0E94B11F6A
:106E20000E940212182F882399F08CE291E00E94B0
:106E3000E321882369F080912B018F5F80932B01E0
:106E4000833118F08AE080932B0181E08093F80071
:106E50008091B706882381F0112371F080912B0176
:106E600060E070E040E050E020E830E00EE210E04A
:106E7000FCE0EF2E0E94B11F0E940212882391F5C0
:106E8000CE0101960E948A1010E08A819B818D5765
:106E90009140A0F011E083E391E00E94E321882378
:106EA00069F080913201813021F482E080933201D7
:106EB00002C01093320181E08093F8008091B70600
:106EC000882381F0112371F08091320160E070E03D
:106ED00040E050E02EE730E00CE210E0ECE0EE2E77
:106EE0000E94B11F0E94132A0E94512B0E94442D20
:106EF0000E948C2E0E942F22A4960FB6F894DEBF1B
:106F00000FBECDBFCF91DF911F910F91FF90EF90FA
:106F1000DF90CF90BF90AF909F908F907F906F90B9
:106F20005F904F903F90089587E06ECF7F928F9251
:106F30009F92AF92BF92CF92DF92EF92FF920F9308
:106F40001F93DF93CF93CDB7DEB760970FB6F8945A
:106F5000DEBF0FBECDBF0E94C922DE011496E8E15C
:106F6000F2E086E001900D928150E1F786E59CE128
:106F70000E94A32880E00E945B118E010C5F1F4FCE
:106F8000C8010E94CC21DD24F02EC12E0CE1A02EE0
:106F9000B12C3BC08091B706882389F180E060E086
:106FA00070E040E050E020E830E00CE210E0EE2439
:106FB0000E94B11F27E22D1510F180E060E070E023
:106FC00040E050E020E830E00E94B11F0D2D10E0BD
:106FD000C501801B910B60E070E040E150E02FE2C2
:106FE00030E00E947F1EC8018C5A9F4F60E070E025
:106FF00040E150E02FE230E00E947F1ED3940E94D7
:10700000132A0E94512B0E941F138F2D9C2D0E942A
:10701000C421882309F4BECF83E00E94C41181E01B
:107020000E94F5110E9492128E01065F1F4FC80147
:107030000E943F11C8010E94AF19882309F08EC039
:107040008F2D9C2DDC01EEE1F2E086E001900D92A7
:107050008150E1F713E0F12E4E010894811C911C40
:10706000B4E0AB2EB12CAC0EBD1E77247394C401DA
:107070000E948A10C5010E94E321882381F081E0EB
:10708000F81619F0FF24F39408C08981882319F4B5
:10709000A3E0FA2E02C0F2E0FF2E7092F800809179
:1070A000B7068823C1F10E94EC2282E89CE10E948D
:1070B00025230E94E9226C0180E060E070E045E059
:1070C00050E020E730E009E110E0E3E0EE2E0E941E
:1070D0007D208F2D60E770E040E050E02FE030E051
:1070E00006E110E0EE240E94B11F83E090E06AE127
:1070F00070E04AE750E02EE030E00E94FF1E498138
:1071000050E0440F551F85E090E06CE170E02AE00C
:1071100030E00E943F1E0E94DA290E94FB230E9459
:1071200023240E94132A0E948C2E0E94512B0E941D
:10713000442D0E941F130E946912882331F08A8116
:107140009B818050904809F492CF8DE00E945B11A2
:1071500083E00E94C41181E00E94F5118091C6066F
:107160000E94AA2882E191E062E070E00E94F12191
:1071700060960FB6F894DEBF0FBECDBFCF91DF9102
:107180001F910F91FF90EF90DF90CF90BF90AF9045
:107190009F908F907F900895991B79E004C0991F6C
:1071A000961708F0961B881F7A95C9F78095089561
:1071B000AA1BBB1B51E107C0AA1FBB1FA617B7071D
:1071C00010F0A61BB70B881F991F5A95A9F7809539
:1071D0009095BC01CD01089597FB092E07260AD092
:1071E00077FD04D0E5DF06D000201AF47095619594
:1071F0007F4F0895F6F7909581959F4F0895DC0194
:10720000CB01FC01E199FECF06C0FFBBEEBBE09ACB
:1072100031960DB20D9241505040B8F70895E19962
:10722000FECF9FBB8EBBE09A99278DB30895DC01FA
:10723000A40FB51F4150504048F0CB01840F951F5B
:107240002E910E94283941505040D0F70895262FA2
:10725000E199FECF9FBB8EBBE09A01970DB202165B
:1072600031F02DBB0FB6F894E29AE19A0FBE089563
:04727000F894FFCFC0
:10727400787878003A00780000800600000101DA8E
:10728400070101008001FF00000000012C01010042
:1072940000008001684201000001640F0101301DFB
:1072A4001E0203A21D0300000000000000000000F5
:1072B40000000000000000000000000000000000CA
:1072C40000000000000000000000000000000000BA
:1072D40000000000000000000000000000000000AA
:1072E400000000000000000000000000000000009A
:1072F400000000000000000000000000000000008A
:10730400010080010000008001010108000100006B
:1073140000000001000001008001000000010001E4
:10732400000000008001000001004D000100000188
:1073340064000100000100000100000A0153000183
:1073440000000101F40101000000800001000100BF
:107354000001140001000000008001000000800111
:10736400320001000001A00F010000010204080A1C
:107374001428505C01097701017A01028001038914
:107384000108A10103AA0103B30103BC0103C50160
:1073940003CE0108E60108FE01030702010A020503
:1073A400190201FFFFFFFFFFFFFF000302050003B7
:1073B400050104060204000103070F1F3F7F0F00AD
:1073C400010500050000000600000101DA070014B1
:1073D4000001050001010904040506070708070662
:1073E40005013200010000000A0001000017171710
:1073F40017171718191A1B1C1D1E1F2021222324BE
:107404002526272828280404050607070807060553
:10741400010000010000000F00010000000F000146
:107424000000000F0001000001701701000001F4CA
:047434000101000052
:00000001FF
